:060000000CEF00F001000E
:0E0006001200D8CFFFF5FACFFEF5BBEF12F0D7
:10001800400EE96E000EEA6EFE0EE16E020EE26E12
:10002800CBEC33F0770EE96E050EEA6EE20EE16E68
:10003800050EE26ECBEC33F0C60EE96E000EEA6EEA
:10004800000EE16E010EE26E840EF66E000EF76E83
:10005800000EF86EC3EC33F0760EE96E050EEA6E0C
:10006800770EE16E050EE26E040EF66E000EF76E68
:10007800000EF86EC3EC33F00FEF13F02707E0061D
:100088004E0700079B0984096809AD091E0AFD0986
:10009800C5094B09570A480A430A4D0A3E0A520A3B
:1000A8005C0ACE0A680A810A0D0BA30AB90AF20A89
:1000B800E60A8B0A780A0ED00101006F3F0EC716B8
:1000C800C66AC56AC686C75094869488C68A00518F
:1000D800C86E1200F1D7850197D085C187F186C116
:1000E80088F10101896F00D01F0E006E0050C51401
:1000F800006E016A000EC7B4010E0010026E0150B6
:10010800036E03500210D8A401D001D0EDD7C580EA
:1001180000D0C5B001D001D0FCD7A1A601D001D034
:1001280002D0010E70D00101895112DA0009D8B449
:1001380001D001D002D0010E66D000D01F0E006E93
:100148000050C514006E016A000EC7B4010E0010FD
:10015800026E0150036E03500210D8A401D001D0E2
:10016800EDD7C5BC01D001D04CD0880EE96E010E88
:10017800EA6EEF50EDD90009D8B401D001D002D011
:10018800010E41D000D01F0E006E0050C514006E45
:10019800016A000EC7B4010E0010026E0150036E12
:1001A80003500210D8A401D001D0EDD7870EE96E14
:1001B800010EEA6EEF50CCD90009D8B401D001D0B5
:1001C80002D0010E20D000D01F0E006E0050C514C2
:1001D800006E016A000EC7B4010E0010026E0150D5
:1001E800036E03500210D8A401D001D0EDD7C5BCCE
:1001F80001D001D003D0000E06D002D0020E03D0E9
:1002080002D0020E00D0120068D7810164D001012B
:10021800846F81C185F182C186F184515DDF01015E
:10022800836F83510009D8B401D001D002D0835123
:1002380051D006D90101836F83510009D8B401D088
:1002480001D002D0835146D000D01F0E006E00505E
:10025800C514006E016A000EC7B4010E0010026ECC
:100268000150036E03500210D8A401D001D0EDD77D
:10027800C58000D0C5B001D001D0FCD7A1A601D05F
:1002880001D002D0010E26D00101842961D90009CC
:10029800D8B401D001D002D0010E1CD000D01F0E5E
:1002A800006E0050C514006E016A000EC7B4010E3E
:1002B8000010026E0150036E03500210D8A401D042
:1002C80001D0EDD7C5BC01D001D002D0000E02D0BC
:1002D800020E00D012009BD73DD001012B6F00D039
:1002E8001F0E006E0050C514006E016A000EC7B4E0
:1002F800010E0010026E0150036E03500210D8A4C4
:1003080001D001D0EDD701012B5122D90009D8B471
:1003180001D001D002D0010E1CD000D01F0E006EFB
:100328000050C514006E016A000EC7B4010E00101B
:10033800026E0150036E03500210D8A401D001D000
:10034800EDD7C5BC01D001D002D0000E02D0020EFC
:1003580000D01200C2D71DD000D01F0E006E005072
:10036800C514006E016A000EC7B4010E0010026EBB
:100378000150036E03500210D8A401D001D0EDD76C
:10038800C58400D0C5B401D001D0FCD7000E00D080
:100398001200E2D710D0F0D800D0C5B601D001D0F5
:1003A800FCD7C59AC58800D0C5B801D001D0FCD704
:1003B800C95000D01200EFD716D0DED800D0C5B68D
:1003C80001D001D0FCD7C58AC58800D0C5B801D0F6
:1003D80001D0FCD7C58400D0C5B401D001D0FCD76A
:1003E800000E00D01200E9D77A0129D00101806FF0
:0803F8007AC181F17BC182F1A1
:10040000805108DF01017F6F7F510009D8B401D00E
:1004100001D002D07F5116D009D0C0DF7CC1E9FFE6
:100420007DC1EAFFEF6E01017C4B7D2B01017E0750
:100430007E29D8A401D001D0F0D7C2DF01017F6F9F
:100440007F5100D01200D6D723D000D01F0E006EEF
:100450000050C514006E016A000EC7B4010E0010F2
:10046000026E0150036E03500210D8A401D001D0D7
:10047000EDD7C58400D0C5B401D001D0FCD7A1A66A
:1004800001D001D002D0010E02D0000E00D0120027
:10049000DCD761D001012C6F00D01F0E006E005020
:1004A000C514006E016A000EC7B4010E0010026E82
:1004B0000150036E03500210D8A401D001D0EDD733
:1004C000C58000D0C5B001D001D0FCD7A1A601D015
:1004D00001D003D0010E3ED02ED001012C513CD8CA
:1004E0000009D8B401D001D002D0010E33D000D021
:1004F0001F0E006E0050C514006E016A000EC7B4D6
:10050000010E0010026E0150036E03500210D8A4B9
:1005100001D001D0EDD7A1A601D001D002D0010EAB
:1005200019D0C5BC01D001D003D001012B6B03D081
:100530000101040E2B6FC58400D0C5B401D001D0D9
:10054000FCD7A1A601D001D002D0010E03D0010139
:100550002B5100D012009ED712D0C96E01018A6FB4
:10056000C6AE01D001D003D0FF0E08D007D000D016
:10057000C7B001D001D0FCD7000E00D01200EDD7DB
:1005800009D0C58600D0C7A001D001D0FCD7C95082
:1005900000D01200F6D7066A046A056A02500310FA
:1005A00003E1006A016A000C1F0E0612D890062AA9
:1005B00002360336FCE3033202320250005C035081
:1005C000015804E3016E0250005ED88004360536FF
:1005D000062E06BAF0D706AE05D0041E042AD8B4FB
:1005E0000506051E0450026E0550036E06AC000C95
:0C05F000001E002AD8B40106011E000CF9
:100600005458540048544D00474946004347490058
:100610004A504700434C4100574156007465787476
:100620002F706C61696E0000000000000000000087
:10063000746578742F68746D6C0000000000000011
:1006400000000000696D6167652F67696600000042
:100650000000000000000000746578742F68746D5D
:100660006C0000000000000000000000696D616780
:10067000652F6A7065670000000000000000000040
:100680006170706C69636174696F6E2F6A61766105
:100690002D766D00617564696F2F782D77617665B1
:1006A0000000000000000000485454502F312E304C
:1006B00020323030204F4B0D0A436F6E74656E74DC
:1006C0002D747970653A20000D0A0D0A00474554D3
:1006D00000504F535400494E4445582E48544D0045
:1006E000485454502F312E3020323030204F4B0D93
:1006F0000A436F6E74656E742D747970653A2000CC
:10070000485454502F312E3020353033200D0A0DEF
:100710000A5365727669636520556E617661696C0E
:1007200061626C650D0A00485454502F312E302000
:10073000343034204E6F7420666F756E640D0A0D70
:100740000A4E6F7420666F756E642E0D0A000D0AD6
:100750000D0A004D434850537461636B2076322E6E
:100760003000426F6172642053657475702E2E2EB6
:100770000020202020202020202020202020202099
:100780002000434F4D4D414E44532E4347490049AD
:100790004E4445582E48544D00667470006D696390
:1007A000726F63686970000D0A0D0A0D4D43485061
:1007B000537461636B2044656D6F204170706C6988
:1007C000636174696F6E2076312E3020284D696325
:1007D000726F63686970205443502F4950205374DE
:1007E00061636B20322E30290D0A0D0A09313A203F
:1007F0004368616E676520426F6172642073657241
:1008000069616C206E756D6265722E0D0A09323A4F
:10081000204368616E67652064656661756C74204D
:10082000495020616464726573732E0D0A09333A6E
:10083000204368616E67652064656661756C74202D
:100840006761746577617920616464726573732E82
:100850000D0A09343A204368616E67652064656655
:1008600061756C74207375626E6574206D61736B55
:100870002E0D0A09353A20456E61626C65204448A8
:100880004350202620495020476C65616E696E6791
:100890002E0D0A09363A2044697361626C65204462
:1008A000484350202620495020476C65616E696E90
:1008B000672E0D0A09373A20446F776E6C6F6164BA
:1008C000204D50465320696D6167652E0D0A093829
:1008D0003A2053617665202620517569742E0D0AE1
:1008E0000D0A456E7465722061206D656E7520631A
:1008F000686F6963652028312D38293A20000D0A78
:10090000496E76616C696420696E707574207265D9
:10091000636569766564202D20496E707574206961
:10092000676E6F7265642E0D0A5072657373206175
:100930006E79206B657920746F20636F6E74696EB9
:1009400075652E2E2E0D0A002575000D0A4E6F7747
:100950002072756E6E696E67206170706C6963617C
:1009600074696F6E2E2E2E000D0A44656661756CDB
:10097000742047617465776179204164647265739E
:10098000732028000D0A44656661756C7420495017
:1009900020416464726573732028000D0A536572E8
:1009A00069616C204E756D6265722028000D0A44E5
:1009B000656661756C74205375626E6574204D6157
:1009C000736B2028000D0A526561647920746F20D2
:1009D000646F776E6C6F6164204D50465320696D73
:1009E000616765202D2055736520586D6F64656DB6
:1009F0002070726F746F636F6C2E0D0A000D0A44C5
:100A0000484350202620495020476C65616E696E2E
:100A1000672064697361626C65642E0D0A000D0ABB
:100A200044484350202620495020476C65616E6938
:100A30006E6720656E61626C65642E0D0A00504F12
:100A40005254005155495400504153530053544F90
:100A5000520041424F52005553455200323230202D
:100A600052656164790D0A00323330204C6F67673C
:100A7000656420696E0D0A00323030206F6B0D0AFC
:100A800000323231204279650D0A0032323620546C
:100A900072616E7366657220436F6D706C6574650C
:100AA0000D0A00353032204E6F7420696D706C6510
:100AB0006D656E7465640D0A00353330204C6F67C8
:100AC000696E2072657175697265640D0A00333351
:100AD000312050617373776F72642072657175692C
:100AE0007265640D0A0031323520446F6E652E0D3B
:100AF0000A00313530205472616E73666572726916
:100B00006E6720646174612E2E2E0D0A0035303020
:100B1000200D0A00D96AD950220D100EF324E16E7F
:100B2000020EF420E26EE76A210EE124E96E000E67
:100B3000E220EA6EEF50FE0BEF6E210EE124E96E2B
:100B4000000EE220EA6EEF50FD0B0209EF6E210E5F
:100B5000E124E96E000EE220EA6EEF50FB0B04097F
:100B6000EF6E210EE124E96E000EE220EA6EEF50F6
:100B7000EF0BEF6E210EE124E96E000EE220EA6E2B
:100B8000EF50F70BEF6E0F0EE124E96E000EE2203E
:100B9000EA6EFF0EEF6E1F0EE124E96E000EE220FA
:100BA000EA6E580EEE6E020EED6ED92A070ED95C73
:100BB000D8A0B1D70201006B040E016F0201046BD3
:100BC000056B066B076B12000101D96AD950220D23
:100BD000100EF324E16E020EF420E26EE750D8A46A
:100BE00047D0010EE76E0B0EE124E96E000EE22005
:100BF000EA6E01C1EEFF02C1EDFF0D0EE124E96EC8
:100C0000000EE220EA6EEE6AED6A070EE124E96E5C
:100C1000000EE220EA6EEE6AEE6AEE6AED6AED52CE
:100C2000ED52210EE124E96E000EE220EA6EEF5053
:100C3000FE0B0109EF6E210EE124E96E000EE220A9
:100C4000EA6EEF50F70BEF6E0F0EE124E96E000E27
:100C5000E220EA6EFF0EEF6E210EE124E96E000E37
:100C6000E220EA6EEF50FD0B0209EF6ED950120040
:100C7000D92A070ED95CD8B0FE0CA8D7D96A0101D1
:100C80000B6B01010B51220D100EF324E16E020ECD
:100C9000F420E26EE750D8A403D0D96AD92A06D04E
:100CA00001010B2B070E0B5DD8A0EBD7D950D8B4A0
:100CB000FE0C0201002B000E01230B0EE124E96E55
:100CC000000EE220EA6E00C2EEFF01C2EDFF130E3D
:100CD000015D890ED8B4005DD8A003D0006B040E6E
:100CE000016F210EE124E96E000EE220EA6EEF5062
:100CF000FE0BEF6E0D0EE124E96E000EE220EA6EAF
:100D000009C1EEFF0AC1EDFF0201042B000E05230D
:100D100006230723140EE124E96E000EE220EA6E9A
:100D200004C2EEFF05C2EEFF06C2EEFF07C2EEFFF1
:100D3000180EE124E96E000EE220EA6EEE6AEE6A19
:100D4000EE6AED6AED52ED52010EE124E8CF46F174
:100D5000000EE220E8CF47F1E1CF0CF1E2CF0DF138
:100D600007C148F108C149F101010A0E4A6F4B6BF6
:100D7000F7EC32F00CC1E1FF0DC1E2FF010EE124FE
:100D8000E8CF70F1000EE220E8CF71F10B0EE12404
:100D9000E96E000EE220EA6EEECF00F0EDCF01F03A
:100DA00000C072F101C073F10D0EE124E96E000E76
:100DB000E220EA6EEECF00F0EDCF01F000C074F15A
:100DC00001C075F1140EE124E96E000EE220EA6E16
:100DD000EECF76F1EECF77F1EECF78F1EDCF79F17E
:100DE000ED52ED52180EE124E96E000EE220EA6E9B
:100DF000EECF7AF1EECF7BF1EECF7CF1EDCF7DF14E
:100E0000ED52ED52020EE8CF7EF1FF0EE8CF7FF1FA
:100E10000101806B816B37EC0BF00CC1E1FF0DC160
:100E2000E2FF030EE76E140EE124E96E000EE220ED
:100E3000EA6EEE2A000EEE22EE22ED22ED52ED5287
:100E400001010B511200D96E220D100EF324E96E30
:100E5000020EF420EA6EEF50040A000ED8B4010E20
:100E60001200D96E220D100EF324E16E020EF42052
:100E7000E26ED9500101666FE1CF67F1E2CF68F110
:100E8000E750040AD8B406D067C169F168C16AF1B5
:100E90002DEF0EF001016651FFD967C1E1FF68C176
:100EA000E2FF010EE124E8CF70F1000EE220E8CF6E
:100EB00071F10B0EE124E96E000EE220EA6EEECF36
:100EC00000F0EDCF01F000C072F101C073F10D0E22
:100ED000E124E96E000EE220EA6EEECF00F0EDCFE5
:100EE00001F000C074F101C075F1140EE124E96E47
:100EF000000EE220EA6EEECF76F1EECF77F1EECF84
:100F000078F1EDCF79F1ED52ED52180EE124E96E52
:100F1000000EE220EA6EEECF7AF1EECF7BF1EECF5B
:100F20007CF1EDCF7DF1ED52ED52110EE8CF7EF167
:100F3000FF0EE8CF7FF10101806B816B98DB67C109
:100F4000E1FF68C1E2FF140EE124E96E000EE22029
:100F5000EA6EEE2A000EEE22EE22ED22ED52ED5266
:100F6000050EE76E1200D96E220D100EF324E16E0D
:100F7000020EF420E26E0F0EE124E96E000EE22074
:100F8000EA6EEF50006E0028D8B4000C210EE12468
:100F9000E96E000EE220EA6EEF50006E00A2000C37
:100FA000010EE124E8CF70F1000EE220E8CF71F1EC
:100FB0000B0EE124E96E000EE220EA6EEECF00F0A7
:100FC000EDCF01F000C072F101C073F10D0EE1240C
:100FD000E96E000EE220EA6EEECF00F0EDCF01F0F8
:100FE00000C074F101C075F1140EE124E96E000E29
:100FF000E220EA6EEECF76F1EECF77F1EECF78F128
:10100000EDCF79F1ED52ED52180EE124E96E000EAC
:10101000E220EA6EEECF7AF1EECF7BF1EECF7CF1FB
:10102000EDCF7DF1ED52ED52100EE8CF7EF10F0EB7
:10103000E124E96E000EE220EA6EEF50E8CF7FF186
:10104000100EE124E96E000EE220EA6EEECF00F011
:10105000EDCF01F000C080F101C081F1E1CF6EF170
:10106000E2CF6FF104DB6EC1E1FF6FC1E2FF140E4E
:10107000E124E96E000EE220EA6EEECF0CF2EECF34
:101080000DF2EECF0EF2EDCF0FF2ED52ED52100E4B
:10109000E124E96E000EE220EA6EEECF00F0EDCF23
:1010A00001F000C002F201C003F2100EE124E96E6B
:1010B000000EE220EA6EEECF00F0EDCF01F0140E4C
:1010C000E124E96E000EE220EA6E0050EE260150A7
:1010D000EE22000EEE22ED22ED52ED52140EE1242E
:1010E000E96E000EE220EA6EEECF0CF2EECF0DF2CA
:1010F000EECF0EF2EDCF0FF2ED52ED52210EE124C4
:10110000E96E000EE220EA6EEF50FD0BEF6E210E4D
:10111000E124E96E000EE220EA6EEF50EF0BEF6E75
:1011200001010F0E6E25E96E000E6F21EA6EEF5081
:10113000C7EC26F06EC1E1FF6FC1E2FF0F0EE124A4
:10114000E96E000EE220EA6EFF0EEF6E210EE12442
:10115000E96E000EE220EA6EEF50FD0B0209EF6E21
:10116000010CD96E220D1F0EF324E96E020EF4203D
:10117000EA6EEF50006E0028D8B4C3EF25F0D950C6
:10118000220D310EF324E96E020EF420EA6EEF30E8
:10119000010B12006A01D96E220D100EF324010119
:1011A0006C6F020EF4206D6FD9506B6F0F0E6C25B3
:1011B000E96E000E6D21EA6EEF50006E0028D8A493
:1011C00027D00F0E6C25E96E000E6D21EA6EEF6AD6
:1011D0000F0E6C25E96E000E6D21EA6EEF50F1ECFA
:1011E00026F00101100E6C25E96E000E6D21EA6EED
:1011F000EE6AED6A0101280EA86FA96B01010F0EBE
:101200006C25E96E000E6D21EA6EEF50ECEC26F0D5
:101210000101100E6C25E96E000E6D21EA6EEECF15
:10122000F3FFEDCFF4FF000EF45CC40ED8B4F35C12
:10123000D8B0000C210E6C25E96E000E6D21EA6E0F
:10124000EF50EF0B1009EF6E6A5176EC26F06CC18F
:10125000E1FF6DC1E2FF100EE124E96E000EE22015
:10126000EA6EEECFF3FFEDCFF4FFF34AF42A100E4F
:10127000E124E96E000EE220EA6EF3CFEEFFF4CF38
:10128000EDFF000EF45CC40ED8B4F35CD8A0010CE2
:1012900001016B5168DE010CD96E220D100EF32492
:1012A000E16E020EF420E26EE1CF69F1E2CF6AF165
:1012B000210EE124E96E000EE220EA6EEF50006E8E
:1012C00000A6000C53EC26F00101210E6925E96E01
:1012D000000E6A21EA6EEF50F70BEF6E010C000171
:1012E000D96E220D100EF324E16E020EF420E26E90
:1012F000210EE124E96E000EE220EA6EEF50006E4E
:1013000000A633D0E1CF00F1E2CF01F1210EE124BC
:10131000E96E000EE220EA6EEF50006E00A410D0DD
:101320000101280E6A6F6B6BD0EC26F00101210ED3
:101330000025E96E000E0121EA6EEF50FB0BEF6E07
:101340000101210E0025E96E000E0121EA6EEF5029
:10135000EF0B1009EF6E00C140F101C141F102C174
:1013600042F103C143F139EF26F0006A016A12002D
:101370006601D96E220D100EF324E16E020EF420E8
:10138000E26E210EE124E96E000EE220EA6EEF50DB
:10139000006E00A6000CE1CF68F1E2CF69F1210EEA
:1013A000E124E96E000EE220EA6EEF50006E00A428
:1013B00010D00101280E6A6F6B6BD0EC26F0010192
:1013C000210E6825E96E000E6921EA6EEF50FB0BD5
:1013D000EF6E0101120E6825E96E000E6921EA6EBA
:1013E000EE50ED10D8A40DD053EC26F00101210EE3
:1013F0006825E96E000E6921EA6EEF50F70BEF6E7B
:10140000000C0101120E6825E96E000E6921EA6EDA
:10141000EE06000EED5A0FEC26F066C1E9FF67C13B
:10142000EAFFEF6E010CD96E220D310EF324E96E46
:10143000020EF420EA6EEF30006E00320030010B35
:101440001200120006010101190E406F010E416FDA
:101450000101140E426F436B39EC26F00101190EA5
:10146000A86F010EA96F32DB0101060E0625E96E99
:10147000000E0721EA6EEECF0DF1EECF0EF1EECFAA
:101480000FF1EDCF10F1ED52ED527BC011F17CC0A8
:1014900012F17DC013F17EC014F1156B060EE8CF7A
:1014A00016F108C117F109C118F117C1C3F118C12C
:1014B000C4F1E9EC2BF000C017F101C018F10101F3
:1014C0000D0EC16F010EC26F01010C0EC36FC46B14
:1014D00052EC2CF0001C026E011C036E02C00BF1DA
:1014E00003C00CF10101240E6A6F6B6BD0EC26F087
:1014F0000B0EE96E010EEA6EEF5076EC26F00C0E44
:10150000E96E010EEA6EEF5076EC26F00101140E42
:101510006A6F6B6BD0EC26F008C1A8F109C1A9F184
:10152000B2D900C00BF101C00CF1290EE96E010E19
:10153000EA6E0101EE520C51ED18D8B40BC1E8FF70
:10154000EF18D8B403D053EC26F0010C0101253973
:101550000F0B006ED8900036D8900034EC0FD96E87
:10156000085D006E0951D8A00905016EEC0E00243B
:10157000086FFF0E0120096F25390F0B006E016AFD
:10158000D89000360136D89000360136140E00246B
:10159000E8CF6AF1000E0120E8CF6BF1D0EC26F025
:1015A0000101190E2D6F010E2E6F06C12FF107C11B
:1015B00030F1BBD901010A6FFE0E0A5DD8A045D0FB
:1015C00053EC26F001010A29D8A4010C08C100F04F
:1015D00009C101F0026A036A005021270150222349
:1015E000025023230350242326B302D026A106D081
:1015F0000101212B000E22232323242306C170F195
:1016000007C171F11BC172F11CC173F119C174F1F1
:101610001AC175F121C176F122C177F123C178F1A8
:1016200024C179F11DC17AF11EC17BF11FC17CF18A
:1016300020C17DF1040EE8CF7EF1FF0EE8CF7FF1EF
:101640000101806B816B13D8010C06C12DF107C11C
:101650002EF10101190E2F6F010E306F08C131F10B
:1016600009C132F101010A517CDB010C7001C3ECAC
:1016700025F00009D8B4FBD772C194F173C195F17C
:1016800074C196F175C197F176C198F177C199F15E
:1016900078C19AF179C19BF17AC19CF17BC19DF12E
:1016A0007CC19EF17DC19FF10101A1513F0BA16F52
:1016B000A051F00BA06F7EC1A1F1F2EC26F000C0AA
:1016C000A2F101C0A3F10101000EA35D290ED8B45F
:1016D000A25DD8A005D0D80EA227FF0EA32303D069
:1016E0000101A26BA36B0101A46BA56BA66BA76B99
:1016F0000101940EA86F010EA96FE8D9140E010123
:101700008027000E81237EA312D0040E8027000EB6
:101710008123020EE8CF84F1040EE8CF85F1866BB9
:10172000FA0EE8CF87F1A0510F0B600904D0010138
:10173000A0510F0B5009A06F7BC088F17CC089F1CC
:101740007DC08AF17EC08BF10101060E7025E96E25
:10175000000E7121EA6EEECF8CF1EECF8DF1EECF5F
:101760008EF1EDCF8FF1ED52ED52906B060EE8CF7A
:1017700091F180C192F181C193F192C1C3F193C102
:10178000C4F1E9EC2BF000C092F101C093F101012A
:10179000880EC16F010EC26F01010C0EC36FC46BC6
:1017A00052EC2CF0001C026E011C036E02C0A4F16E
:1017B00003C0A5F1A40EE96E010EEA6EEECF82F130
:1017C000EDCF83F101017F29D8B47F6B0101140EA5
:1017D000A86FA96B01017F51ECEC26F070C1A8F154
:1017E00071C1A9F1060EE8CFAAF180C1ABF181C1A8
:1017F000ACF1B5EC29F00101940EC16F010EC26F7E
:101800000101140EC36FC46BA0EC26F07EA30BD0B5
:101810000101840EC16F010EC26F0101040EC36F7E
:10182000C46BA0EC26F00101140EA86FA96B010196
:101830007F51ECEC26F080C1A8F181C1A9F123D839
:1018400000C082F101C083F10101240EA86FA96BD1
:1018500001017F51ECEC26F0830EE96E010EEA6E79
:10186000EF5076EC26F0820EE96E010EEA6EEF5034
:1018700076EC26F00101A86BA96B01017F51ECEC1D
:1018800026F0BCEF26F00101AA6BAA2BAC6BAD6B66
:101890000101A951016EA851006EA807D8A0A9079F
:1018A0000110D8B42CD00FEC26F00101AB6FAA5177
:1018B000D8A40FD0AB51AC25E8CFACF1AB51ACC143
:1018C00000F0005CD8B014D0AD3F12D00101AC2BB9
:1018D0000FD00101AB51AD25E8CFADF1AB51ADC19A
:1018E00000F0005CD8B004D0AC3F02D00101AD2BB9
:1018F0000101AA51000ED8B4010EAA6FC9D7AD0ECE
:10190000E96E010EEA6EEF50FF0AE8CFADF1AC0EC2
:10191000E96E010EEA6EEF50FF0AE8CFACF1ACC100
:1019200000F0ADC101F012002D010101FE0E316F7A
:10193000016A0150220D100EF324D96E020EF4201C
:10194000DA6EDF50D8B44ED00101020E2D25E16EC3
:10195000000E2E21E26E0B0ED924E96E000EDA2065
:10196000EA6EEE52E652E550ED18E7CFE8FFD8B444
:10197000EF18D8A437D0DF50006E0004D8A402D0EE
:101980000150316F2DC1E9FF2EC1EAFF0D0ED924A0
:10199000E16E000EDA20E26EE652EE52ED50E518EE
:1019A000EFCFE8FFD8B4E718D8A41CD00101060E89
:1019B0002F25E16E000E3021E26E070ED924E96E6C
:1019C000000EDA20EA6EEE50E61808E1EE50E61856
:1019D00005E1EE50E61802E1EE50E618D8A402D078
:1019E00001501200012A070E015CD8A0A2D7010104
:1019F0003151220D100EF324E16E020EF420E26E3E
:101A00003151FE0AD8B45BD0E750006E0004D8A470
:101A100056D0010EE124E8CF46F1000EE220E8CFD7
:101A200047F1E1CF32F1E2CF33F12FC148F130C1BC
:101A300049F101010A0E4A6F4B6BF7EC32F032C1EB
:101A4000D9FF33C1DAFF0101020E2D25E16E000E30
:101A50002E21E26E0B0ED924E96E000EDA20EA6E1A
:101A6000E6CFEEFFE5CFEDFF2DC1E9FF2EC1EAFF86
:101A70000D0ED924E16E000EDA20E26EEECFE6FF05
:101A8000EDCFE5FF210ED924E96E000EDA20EA6ED3
:101A9000EF50F70BEF6E0F0ED924E96E000EDA202F
:101AA000EA6EFF0EEF6E210ED924E96E000EDA20E9
:101AB000EA6EEF50FD0B0209EF6E31511200010189
:101AC0003151FE0AD8B4FF0CFE0CA801A8C1E9FFF1
:101AD000A9C1EAFFEECF00F0EDCF01F000C0C3F1E5
:101AE00001C0C4F1E9EC2BF0A8C1E9FFA9C1EAFFEC
:101AF00000C0EEFF01C0EDFF0101020EA825E96E56
:101B0000000EA921EA6EEECF00F0EDCF01F000C08B
:101B1000C3F101C0C4F1E9EC2BF00101020EA825CC
:101B2000E96E000EA921EA6E00C0EEFF01C0EDFFD4
:101B3000040EA825E96E000EA921EA6EEECFAAF1E7
:101B4000EECFABF1EECFACF1EDCFADF1ED52ED520A
:101B500000EC2CF00101040EA825E96E000EA9216D
:101B6000EA6E00C0EEFF01C0EEFF02C0EEFF03C050
:101B7000EEFF080EA825E96E000EA921EA6EEECF51
:101B8000AAF1EECFABF1EECFACF1EDCFADF1ED526E
:101B9000ED5200EC2CF00101080EA825E96E000EB4
:101BA000A921EA6E00C0EEFF01C0EEFF02C0EEFF09
:101BB00003C0EEFF0E0EA825E96E000EA921EA6E05
:101BC000EECF00F0EDCF01F000C0C3F101C0C4F1D1
:101BD000E9EC2BF001010E0EA825E96E000EA921FB
:101BE000EA6E00C0EEFF01C0EDFF100EA825E96E01
:101BF000000EA921EA6EEECF00F0EDCF01F000C09B
:101C0000C3F101C0C4F1E9EC2BF00101100EA825CD
:101C1000E96E000EA921EA6E00C0EEFF01C0EDFFE3
:101C2000120EA825E96E000EA921EA6EEECF00F093
:101C3000EDCF01F000C0C3F101C0C4F1E9EC2BF01D
:101C40000101120EA825E96E000EA921EA6E00C05E
:101C5000EEFF01C0EDFF1200690101010F0E6925C1
:101C6000E96E000E6A21EA6EEF50006E0028D8B4CB
:101C70001FD00F0E6925E96E000E6A21EA6EEF5043
:101C8000C7EC26F069C1E1FF6AC1E2FF0F0EE12453
:101C9000E96E000EE220EA6EFF0EEF6E210EE124E7
:101CA000E96E000EE220EA6EEF50FD0B0209EF6EC6
:101CB00069C1E1FF6AC1E2FF070EE124E96E000E8F
:101CC000E220EA6EEE6AEE6AEE6AED6AED52ED52DD
:101CD0000D0EE124E96E000EE220EA6E000EEE6ABF
:101CE000ED6AE1CF69F1E2CF6AF1210EE124E96EFC
:101CF000000EE220EA6EEF50006E00B653EC26F0C4
:101D000069C1E1FF6AC1E2FF210EE124E96E000E24
:101D1000E220EA6EEF50F70BEF6E1F0EE124E96E42
:101D2000000EE220EA6E580EEE6E020EED6E210EEF
:101D3000E124E96E000EE220EA6EEF50EF0BEF6E49
:101D4000210EE124E96E000EE220EA6EEF50006EF3
:101D500000A003D0010EE76E1200000EE76A120029
:101D60002D01D96E0101336BD950220D100EF324D1
:101D7000E16E020EF420E26E180EE124E96E000E10
:101D8000E220EA6EEECF36F1EECF37F1EECF38F14A
:101D9000EECF39F1140EE124E96E000EE220EA6E76
:101DA000EECF3AF1EECF3BF1EECF3CF1EECF3DF18D
:101DB000040E2F25E96E000E3021EA6EEECF42F1BF
:101DC000EECF43F1EECF44F1EECF45F131C100F05B
:101DD00032C101F0026A036A0050422701504323D6
:101DE0000250442303504523140EE124E96E000EF3
:101DF000E220EA6EEECF3EF1EECF3FF1EECF40F1C2
:101E0000EECF41F1080E2F25E96E000E3021EA6E6B
:101E1000EECF08F2EECF09F2EECF0AF2EDCF0BF2E1
:101E2000ED52ED521C0EE124E96E000EE220EA6E46
:101E3000000EEF6AE1CF34F1E2CF35F185EC33F0FB
:101E400001011D0E3425E96E000E3521EA6E00C039
:101E5000EEFF01C0EDFF34C1D9FF35C1DAFF1F0E1F
:101E6000D924E96E000EDA20EA6E580EEE6E020EEC
:101E7000ED6EDF50006E0004D8A4A5D053EC26F020
:101E800034C1D9FF35C1DAFF0201042B000E05234E
:101E900006230723140ED924E96E000EDA20EA6E19
:101EA00004C2EEFF05C2EEFF06C2EEFF07C2EEFF60
:101EB0000101422B000E432344234523180ED9244D
:101EC000E96E000EDA20EA6E42C1EEFF43C1EEFF7A
:101ED00044C1EEFF45C1EEFF140ED924E96E000E99
:101EE000DA20EA6EEECF3EF1EECF3FF1EECF40F1D9
:101EF000EECF41F1140ED924E96E000EDA20EA6E1D
:101F0000EE2A000EEE22EE22ED22ED52ED522FC10E
:101F1000E1FF30C1E2FF0D0EE124E96E000EE22088
:101F2000EA6EEF50006E00A229D0010ED924E8CF4E
:101F300046F1000EDA20E8CF47F12DC148F12EC15D
:101F400049F101010A0E4A6F4B6BF7EC32F034C1D4
:101F5000D9FF35C1DAFF2FC1E9FF30C1EAFF0D0E0D
:101F6000D924E16E000EDA20E26EEECFE6FFEDCF6F
:101F7000E5FF0101120E336F020E62D20101040E61
:101F8000336F42C13EF143C13FF144C140F145C10D
:101F900041F1E124E96E000EE220EA6EEECF42F15B
:101FA000EECF43F1EECF44F1EECF45F1070ED92449
:101FB000E96E000EDA20EA6EEE6AEE6AEE6AED6A0B
:101FC000ED52ED5259D22FC1E1FF30C1E2FF0D0EAB
:101FD000E124E96E000EE220EA6EEF50006E00A4EC
:101FE00007D053EC26F034C169F135C16AF135D61A
:101FF000080EE124E96E000EE220EA6E0101EE50C7
:102000003E1908E1EE503F1905E1EE50401902E19A
:10201000EE504119D8A42ED2DF50020AD8A457D0CE
:102020000D0EE124E96E000EE220EA6EEF50006E24
:1020300000A84AD0180ED924E96E000EDA20EA6E04
:1020400042C1EEFF43C1EEFF44C1EEFF45C1EEFFCA
:102050001C0ED924E96E000EDA20EA6E000EEF6A3B
:1020600085EC33F001011D0E3425E96E000E35219B
:10207000EA6E00C0EEFF01C0EDFF34C1E1FF35C1E3
:10208000E2FF040EE76E32513111D8B41AD0210E9E
:10209000E124E96E000EE220EA6EEF50F70B08092A
:1020A000EF6E120EE124E96E000EE220EA6E31C1FD
:1020B000EEFF32C1EDFF210EE124E96E000EE220B9
:1020C0006DD053EC26F0D8D153EC26F0D5D1DF50AB
:1020D000030AD8A46FD00D0EE124E96E000EE220B1
:1020E000EA6EEF50006E00A262D00101422B000E9A
:1020F000432344234523180ED924E96E000EDA2029
:10210000EA6E42C1EEFF43C1EEFF44C1EEFF45C19E
:10211000EEFF0D0EE124E96E000EE220EA6EEF50B4
:10212000006E00A805D0100E336F040EDF6E18D0BD
:102130000101120E336F020EDF6E3E2B000E3F23A5
:1021400040234123140ED924E96E000EDA20EA6EF2
:102150003EC1EEFF3FC1EEFF40C1EEFF41C1EEFFC9
:10216000010132513111D8B41FD0210ED924E96EAA
:10217000000EDA20EA6EEF50F70B0809EF6E120E30
:10218000D924E96E000EDA20EA6E31C1EEFF32C1C9
:10219000EDFF210ED924E96E000EDA20EA6EEF5031
:1021A000FB0B0409EF6E68D153EC26F065D153ECBC
:1021B00026F062D1180ED924E16E000EDA20E26E0C
:1021C0000101040E2F25E96E000E3021EA6EEE505B
:1021D000E61808E1EE50E61805E1EE50E61802E1D7
:1021E000EE50E618D8A453EF26F0180ED924E96E65
:1021F000000EDA20EA6E42C1EEFF43C1EEFF44C199
:10220000EEFF45C1EEFFDF50040AD8A4BFD00101A4
:102210000D0E2F25E96E000E3021EA6EEF50006E94
:1022200000A82AD00F0ED924E96E000EDA20EA6E3B
:10223000EF50006E0028D8B41FD00F0E3425E96E81
:10224000000E3521EA6EEF50C7EC26F034C1D9FFFD
:1022500035C1DAFF0F0ED924E96E000EDA20EA6EDE
:10226000FF0EEF6E210ED924E96E000EDA20EA6E21
:10227000EF50FD0B0209EF6E01010D0E2F25E96EE7
:10228000000E3021EA6EEF50006E00A02BD0110E30
:10229000336F140ED924E96E000EDA20EA6E97EC43
:1022A00033F000C03EF101C03FF102C040F103C075
:1022B00041F1180ED924E96E000EDA20EA6EEE2AFA
:1022C000000EEE22EE22ED22ED52ED52EECF42F163
:1022D000EECF43F1EECF44F1EDCF45F1ED52ED52AB
:1022E0000A0EDF6E010132513111D8B44CD0210EEB
:1022F000D924E96E000EDA20EA6EEF50006E00B6C7
:1023000021D0210ED924E96E000EDA20EA6EEF50BA
:10231000F70B0809EF6E120ED924E96E000EDA20D1
:10232000EA6E31C1EEFF32C1EDFF210ED924E96E14
:10233000000EDA20EA6EEF50FB0B0409EF6E100E70
:10234000336F9AD00101336B140ED924E96E000E5D
:10235000DA20EA6E3AC1EEFF3BC1EEFF3CC1EEFF70
:102360003DC1EEFF180ED924E96E000EDA20EA6EA8
:1023700036C1EEFF37C1EEFF38C1EEFF39C1EEFFC7
:1023800053EC26F079D053EC26F076D0DF500A0AD1
:10239000D8A413D053EC26F001010D0E2F25E96EC1
:1023A000000E3021EA6EEF50006E00A865D034C1F7
:1023B00069F135C16AF151DC5FD0DF50050AD8A45C
:1023C00041D053EC26F02FC1E1FF30C1E2FF0D0EEA
:1023D000E124E96E000EE220EA6EEF50006E00A0EC
:1023E0004BD00101100E336F34C1D9FF35C1DAFF74
:1023F000180ED924E96E000EDA20EA6EEE2A000EDD
:10240000EE22EE22ED22ED52ED52EECF42F1EECF72
:1024100043F1EECF44F1EDCF45F1ED52ED520D0E0B
:10242000E124E96E000EE220EA6EEF50006E00A893
:1024300006D0D9CF69F1DACF6AF10FDC1DD0060ED4
:10244000DF6E1AD0DF50060AD8A416D053EC26F05F
:1024500001010D0E2F25E96E000E3021EA6EEF50BE
:10246000006E00A809D034C169F135C16AF12DECC4
:102470000EF002D053EC26F001013351D8B4120013
:102480002DC170F12EC171F12FC1E1FF30C1E2FF0A
:10249000020EE124E96E000EE220EA6EEECF00F0BB
:1024A000EDCF01F000C072F101C073F1E6CF00F092
:1024B000E5CF01F000C074F101C075F13EC176F1C5
:1024C0003FC177F140C178F141C179F142C17AF160
:1024D00043C17BF144C17CF145C17DF133C17EF143
:1024E000FF0EE8CF7FF10101806B816B37EF0BF0BE
:1024F0008AEC33F03EEC24F0E2C5F3FFE3C5F4FFD1
:10250000E4C5F5FFE5C5F6FFE6C5F7FFE7C5F8FF4B
:10251000E8C500F0E9C501F0EAC502F0EBC503F03B
:10252000ECC504F0EDC505F0EEC506F0EFC507F00B
:10253000F0C508F0F1C509F0F2C50AF0F3C50BF0DB
:10254000F4C50CF0F5C50DF0F6C50EF0F7C5DAFFD1
:10255000F8C5D9FFF9C5E2FFFAC5E1FFFBC5EAFFFF
:10256000FCC5E9FFFDC5E8FFFEC5FAFFFFC5D8FFC2
:102570000FC0E0FF1000E0CF0FF0E8CFFDF5E9CF8E
:10258000FCF5EACFFBF5E1CFFAF5E2CFF9F5D9CFCB
:10259000F8F5DACFF7F50EC0F6F50DC0F5F50CC07D
:1025A000F4F50BC0F3F50AC0F2F509C0F1F508C067
:1025B000F0F507C0EFF506C0EEF505C0EDF504C077
:1025C000ECF503C0EBF502C0EAF501C0E9F500C087
:1025D000E8F5F8CFE7F5F7CFE6F5F6CFE5F5F5CF77
:1025E000E4F5F4CFE3F5F3CFE2F582D7ACA2FED762
:1025F000AD6E12002A012AC1E1FF2BC1E2FFE250B9
:10260000016EE150006EE14AE22A00C0E9FF01C01C
:10261000EAFFEF50D96ED8B41200E8DFF0D7F86ABD
:1026200077DA7BEC33F074EC2AF090DA81BA0CD0D4
:10263000C00EB1EC2FF00101620E2A6F070E2B6F56
:102640001CEC30F0ABEC17F07DEC2EF089EC18F0C0
:1026500081EC1DF085EC2EF0ACEC18F096EC1DF042
:102660000DD99DC500F076C5E8FF0018D8B4F2D7A3
:1026700001017B0E1D6F000E1E6F010EE8CF1FF1D2
:1026800019D876C59DF593C000F000A0E3D7CE0E13
:10269000B1EC2FF00A0E9DC500F0005C9DC5E8FF6F
:1026A000D8B004D0300F3CEC30F0D4D7410F3CEC24
:1026B00030F0D0D701011F51D8B40DD0C00EB1EC0D
:1026C0002FF00101710E2A6F070E2B6F1CEC30F0FA
:1026D000C00EB1EC2FF00101200E2C6F010E2D6FFA
:1026E0000101480E2E6F090E2F6F1DC1E9FF1EC19B
:1026F000EAFFEF50006E016A00C028F101C029F125
:10270000280EE8CF2AF1010EE8CF2BF13EEC21F0A4
:1027100001011F51D8B40BD00101200E2A6F010E08
:102720002B6F05EC30F02E0E3CEC30F008D00101A0
:10273000200E2A6F010E2B6F5EDF2E0E57DF010178
:10274000200E2C6F010E2D6F0101480E2E6F090E09
:102750002F6F0101010E1D25E96E000E1E21EA6E8C
:10276000EF50006E016A00C028F101C029F1280E67
:10277000E8CF2AF1010EE8CF2BF13EEC21F0010168
:102780001F51D8B40BD00101200E2A6F010E2B6F00
:1027900005EC30F02E0E3CEC30F008D00101200E9C
:1027A0002A6F010E2B6F27DF2E0E20DF0101200E76
:1027B0002C6F010E2D6F0101480E2E6F090E2F6F29
:1027C0000101020E1D25E96E000E1E21EA6EEF507A
:1027D000006E016A00C028F101C029F1280EE8CF7F
:1027E0002AF1010EE8CF2BF13EEC21F001011F513F
:1027F000D8B40BD00101200E2A6F010E2B6F05EC0F
:1028000030F02E0E3CEC30F008D00101200E2A6F83
:10281000010E2B6FF0DE2E0EE9DE0101200E2C6F73
:10282000010E2D6F0101480E2E6F090E2F6F010151
:10283000030E1D25E96E000E1E21EA6EEF50006E9C
:10284000016A00C028F101C029F1280EE8CF2AF161
:10285000010EE8CF2BF13EEC21F001011F51D8B45D
:1028600007D00101200E2A6F010E2B6F05EF30F00B
:102870000101200E2A6F010E2B6FBDD6810EC26E94
:10288000640EE8CF00F1010100070029D8A4FBD7AE
:10289000C284C2B4FED7C3CF00F1C4CF01F101019D
:1028A0009E0E2C6F050E2D6F0101480E2E6F090E26
:1028B0002F6F00C102F101C103F1020EE8CF2AF12E
:1028C000010EE8CF2BF13EEC21F0840EC16E890E93
:1028D000C26E640EE8CF00F1010100070029D8A400
:1028E000FBD7C284C2B4FED7C3CF00F1C4CF01F17D
:1028F0000101A60E2C6F050E2D6F0101480E2E6FE3
:10290000090E2F6F00C102F101C103F1020EE8CFE1
:102910002AF1010EE8CF2BF13EEC21F08E0EC16EB4
:102920001200660166C1E1FF67C1E2FFE6CF00F079
:10293000E5CF01F000C0E9FF01C0EAFFEF50D00F82
:10294000D96E3FD0020EE124E96E000EE220EA6E5D
:10295000EECF00F0EDCF01F000C0E9FF01C0EAFFCB
:10296000EF50D00FD96E04D0897606D0897404D088
:10297000D950FAE0010AFAE0E6CF00F0E5CF01F025
:1029800000C076F101C077F10101820E786F070E69
:10299000796F0D0EE8CF7AF10EEC2DF01200E6CF34
:1029A00000F0E5CF01F000C076F101C077F1010140
:1029B0008F0E786F070E796F0A0EE8CF7AF10EEF5F
:1029C0002DF0D950BFE0010AE9E0E9D7E16E66D009
:1029D00089B603D060D089A45ED0300E5DD00101ED
:1029E0006B516A11D8A402D06A6B6B6B9E0E006E9D
:1029F000050E016E01016A510024E96E000E0120EE
:102A0000EA6EEFCFDFFF9E0E006E050E016E6A517B
:102A10000024E96E000E0120EA6EEF50D8A404D025
:102A2000FF0E006E016E120001016A4B6B2B6AC132
:102A300000F06BC101F0120001016B516A11D8A4C2
:102A400002D06A6B6B6BA60E006E050E016E010163
:102A50006A510024E96E000E0120EA6EEFCFDFFF1D
:102A6000A60E006E050E016E6A510024E96E000E7E
:102A70000120EA6EEF50D8A404D0FF0E006E016E64
:102A8000120001016A4B6B2B6AC100F06BC101F0AF
:102A9000120081AAA2D7310EDF6E0ED06CC1D9FF11
:102AA0006DC1DAFFE15094E0010A95E0030A97E076
:102AB000010AC2E0070AEDE0FF0E006E016E12008F
:102AC00006010101990E766F070E776F06C178F146
:102AD00007C179F10101030E7A6F7B6B5AEC32F07A
:102AE00001500010D8A4000C01019D0E766F070E56
:102AF000776F08C178F109C179F10101090E7A6F88
:102B00007B6B5AEC32F001500010D8B4010C000C71
:102B10008E0EC16E030E926E809A89848986F19E14
:102B200078EC2FF0800EB1EC2FF00101530E2A6FDC
:102B3000070E2B6F1CEC30F0200EAC6E900EAB6EBF
:102B40000F0EAF6ED56AF28EF28C12000A0EE8CF2D
:102B50007BF0E8CF7CF0050EE8CF7DF00F0EE8CFDC
:102B60007EF0FF0EE8CF85F0E8CF86F0E8CF87F063
:102B70000001886B0A0EE8CF89F0E8CF8AF0050ED5
:102B8000E8CF8BF00F0EE8CF8CF000017F6B040EC6
:102B9000E8CF80F0A30EE8CF81F00001826B000146
:102BA000836B0001846B930EE96E000EEA6EEF50AA
:102BB000FE0BEF6E01017B0E016F000E026F010133
:102BC000816B826BA00E0AEC01F0CEEC01F00101EA
:102BD000006FE0EC01F001010051550AD8A41AD0B1
:102BE0000101010E816F826BA00E0AEC01F0010160
:102BF000006BCEEC01F001C1E9FF02C1EAFFEF6E0C
:102C00000101014B022B002B190E005DD8A0F1D75A
:102C1000E0EF01F001017B0E1E6F000E1F6F01013E
:102C2000856B866BA00E70EC00F0550E70EC01F019
:102C300001011D6B01011F51016E1E51006E1E4BE3
:102C40001F2B00C0E9FF01C0EAFFEF5070EC01F05C
:102C500001011D2B190E1D5DD8A0ECD7AFEF01F0BF
:102C600001011DC1F6FF1EC1F7FF010E1D27000E59
:102C70001E23050EF76403D00800F55005D0F6CFEB
:102C8000E9FFF7CFEAFFEF50D96E0009D8B4120080
:102C9000ADDCE6D71DC1E1FF1EC1E2FFD96A9EAAE5
:102CA000FED7AE50F36E0D0AD8B40DD0F3500A0A19
:102CB000D8B409D0D92AF3CFE6FFE76A01011F078C
:102CC0001F29D8A4ECD7D95012001D011DC1E1FF66
:102CD0001EC1E2FFE1CF22F1E2CF23F10101216B1E
:102CE000E750D96ED8B437D02E0AD8A429D0E250F4
:102CF000016EE150006EE14AE22A00C0E9FF01C026
:102D0000EAFF000EEF6AE1CF1DF1E2CF1EF122C112
:102D100024F123C125F151EC31F0010121511F258E
:102D2000E96E000E2021EA6E00C0EFFF212B1DC1CD
:102D3000E1FF1EC1E2FFE1CF22F1E2CF23F108D093
:102D4000300ED95CD8A0000C3A0ED95CD8B0000C7B
:102D5000E14AE22AC5D722C124F123C125F151EC71
:102D600031F0010121511F25E96E000E2021EA6E8C
:102D700000C0EFFF2151030A000ED8B4010E12006B
:102D80009EAAFED7AE50D96E310ED95C390ED8A0AE
:102D90001200D95CD8B0390CD9501200E16E0D0E7A
:102DA00025DC0A0E23DCE150006E016AD890003465
:102DB000026E0134036E6C0E0224E96E000E0320D5
:102DC000EA6EEECF00F0EDCF01F000C01DF101C0C2
:102DD0001EF146DFADD00101070E2C6F010E2D6FE5
:102DE0000101480E2E6F090E2F6F8D0EE96E000E39
:102DF000EA6EEECF1BF1EDCF1CF11B0EE8CF2AF1EE
:102E0000010EE8CF2BF13EEC21F00101070E2A6FF5
:102E1000010E2B6FFBEC12F0290EF6EC12F03A0EBD
:102E2000F6EC12F0200EF6EC12F00101070E1D6F09
:102E3000010E1E6F140EE8CF1FF12CDF006E016A29
:102E400001500010D8B44AD00101070E246F010EC2
:102E5000256F51EC31F000C08DF001C08EF08EC0B6
:102E600083F08DC084F012007B0EE96E000E07D057
:102E7000890EE96E000E03D0850EE96E000EEA6E33
:102E8000E9CF1DF1EACF1EF1E9CF01F1EACF02F15E
:102E900001011F6B0FDC290EF6EC12F03A0EF6EC76
:102EA00012F0200EF6EC12F00101070E1D6F010E5C
:102EB0001E6F140EE8CF1FF1EDDE0101070E1D6F2E
:102EC000010E1E6F0101030E1F6F010E206FFEDE4B
:102ED000006E016A01500010D8A40AD00101FE0E54
:102EE0001D6F080E1E6FBCDE9EAAFED7AE501200EC
:102EF00001C1E9FF02C1EAFF03C1EEFF04C1EEFF19
:102F000005C1EEFF06C1EEFF1200930EE96E000E42
:102F1000EA6EEF50FE0B0109EF6E1200930EE96EA0
:102F2000000EEA6EEF50FE0BEF6E120028D072D644
:102F3000E150310A01E14FD7030A96E0010A98E017
:102F4000070A9AE0010AE1E0030AE8E0010AEEE07C
:102F50000F0AEDE012000101A70E1D6F070E1E6F94
:102F60007FDE0EDF0101006F390AD8B402D00051B4
:102F700015DF01010051380AD8B41200ECD7010165
:102F8000206B1E6B81EC2BF000C022F101C023F1FD
:102F90000101246B040E256F85EC33F000C028F18D
:102FA00001C029F185EC33F000C026F101C027F102
:102FB00001012951275D02E12851265DD8A011D0D9
:102FC0002851265D006E29512759016E000E015CC3
:102FD000050ED8B4005C000ED8B0010E006E016A78
:102FE0000FD0FF0E006E016E2851005C026E295159
:102FF0000158036E26510224006E27510320016EF2
:1030000001500010D8B40AD085EC33F000C028F18C
:1030100001C029F1150EF6EC12F089749EBA64D045
:10302000C1D79EAA61D08974AE50D96E01012051DA
:10303000010A1CE0030A20E0010A22E0D904D8A416
:1030400003D0206B202B50D0D950040AD8A40AD02A
:10305000898421EC2BF0060EF6EC12F001011E6BB8
:103060001E2B42D0150EF6EC12F03ED0060ED96E95
:1030700001011F6B020E02D00101030E206F34D03C
:1030800001011F512425E96E000E2521EA6ED9CFDA
:10309000EFFF1F2B810E1F5DD8A026D022C12AF181
:1030A00023C12BF191EC2BF00101060E1D6F216B5A
:1030B000010121512425E96E000E2521EA6EEF5011
:1030C000ACEC2BF00101212B800E215DD8A0F0D7B4
:1030D000D3EC2BF000C022F101C023F101011D51FE
:1030E000F6EC12F00101206B01011E51D8B499D702
:1030F000D968D906D928D8B4010CFBD70F0E57EFE1
:1031000033F0040E57EF33F0200ED96ED92EFED7D0
:1031100012000101006B0101500E016F026BE5EC22
:1031200005F0006E010100510A0D940EF324E96EC2
:10313000000EF420EA6E00C0EFFF00510A0D970E5A
:10314000F324E96E000EF420EA6EEF6A002B050E00
:10315000005DD8B01200DFD70101006B0101005102
:1031600007D80101002B050E005DD8B01200F6D77C
:10317000D96E0A0D940EF3240101096F000EF4209C
:103180000A6F026B022B01010251D8B41200026BCC
:1031900009C1E9FF0AC1EAFFEF5023EC07F000097B
:1031A0000101030ED8A411D20925E96E000E0A21EF
:1031B000EA6E000EEF6A120009C1E9FF0AC1EAFFD8
:1031C000EF5013EC0AF000090101D8B4DDD7026B0F
:1031D000022B056B066B0101000E065D500ED8B484
:1031E000055DD8B01AD00651016E0551006E054B31
:1031F000062B150FE8CF66F1010E0120E8CF67F12D
:1032000009C1E9FF0AC1EAFFEF50B9EC09F0006E0D
:10321000016A01500010D8A4DED70101150E052562
:10322000E96E010E0621EA6E000EEF6A09C1E9FFA0
:103230000AC1EAFFEF504CEC09F00101030E092529
:10324000E96E000E0A21EA6E020EEF6E050E036FA4
:103250000101150E666F010E676F01010B0E686F9D
:10326000010E696F0101030E6A6F010E6B6F0101A0
:10327000090E0925E8CF6CF1000E0A21E8CF6DF1A7
:10328000CCDA0101016F0009D8A47DD7020E035DDD
:10329000D8A012D001010B0E666F010E676F03C13B
:1032A00068F192EC14F00101090E0925E96E000E97
:1032B0000A21EA6E030EEF6E0BC166F10CC167F1D5
:1032C00081EC2AF00101010E0925E96E000E0A21A8
:1032D000EA6E00C0EEFF01C0EDFF09C1E1FF0AC1C7
:1032E000E2FF010EE124E96E000EE220EA6EEE52EA
:1032F000ED50FF0AFF0ED8B4EF18D8A411D0080E75
:10330000E124E96E000EE220EA6E000EEF6E030E7D
:10331000E124E96E000EE220EA6E020EEF6E33D772
:10332000010EE124E96E000EE220EA6EEE50ED108F
:10333000D8A408D0080EE124E96E000EE220EA6E5F
:10334000030EE4D7030EE124E96E000EE220EA6EDC
:103350000B0EE4D709C1E9FF0AC1EAFFEF50B1EC57
:1033600008F000090101D8B40FD7080E0925E96E4D
:10337000000E0A21EA6EEF50006E016AD890003408
:10338000026E0134036EC60E0224E96E000E0320A5
:10339000EA6EEECF07F1EDCF08F1010107C1F6FFAC
:1033A00008C1F7FF010E0727000E0823050EF7647A
:1033B00003D00800F55005D0F6CFE9FFF7CFEAFFBC
:1033C000EF50D96E0009D8B40AD0D9CF6AF109C13B
:1033D000E9FF0AC1EAFFEF50CBEC08F0DED709C1E4
:1033E000E9FF0AC1EAFFEF50B3EC07F0C1D009C111
:1033F000E9FF0AC1EAFFEF50B1EC08F00009010152
:10340000D8B4C2D6026B022B046B0451006E016A61
:103410000050A80FF66E0150F76E060EF722080056
:10342000F550E8CF6AF109C1E9FF0AC1EAFFEF50A0
:10343000CBEC08F00101042B1F0E045DD8A0E5D7EA
:10344000090E0925E96E000E0A21EA6EEF50140DEF
:103450001C0EF324076F060EF420086F010107C14C
:10346000F6FF08C1F7FF010E0727000E0823050E1F
:10347000F76403D00800F55005D0F6CFE9FFF7CF89
:10348000EAFFEF50D96E0009D8B40AD0D9CF6AF15B
:1034900009C1E9FF0AC1EAFFEF50CBEC08F0DED723
:1034A0000101046B01010451006E016A0050C80F54
:1034B000F66E0150F76E060EF7220800F550E8CFC1
:1034C0006AF109C1E9FF0AC1EAFFEF50CBEC08F04D
:1034D0000101042B040E045DD8A0E4D709C1E1FF6B
:1034E0000AC1E2FF090EE124E96E000EE220EA6E55
:1034F000EF50030A070ED8A407D0E124E96E000EAE
:10350000E220EA6E010E06D0E124E96E000EE22010
:10351000EA6E000EEF6E040EE124E96E000EE2206A
:10352000EA6E030EEF6EE124E96E000EE220EA6E11
:10353000010EF4D609C1E9FF0AC1EAFFEF5013EC0E
:103540000AF00009D8B407D009C1E9FF0AC1EAFFAF
:10355000EF504CEC09F009C166F10AC167F148D897
:10356000006E016A01500010D8B40DD621EC2BF08A
:103570000101030E0925E96E000E0A21EA6E090E0B
:10358000CDD609C1E9FF0AC1EAFFEF5023EC07F0ED
:103590000009D8B4F8D509C1E9FF0AC1EAFFEF5024
:1035A000B1EC08F00009D8B4EED509C1E9FF0AC1B1
:1035B000EAFFEF5031EC07F00101030E0925E96E37
:1035C000000E0A21EA6E0A0EA9D60925E96E000E40
:1035D0000A21EA6EEF5001E1EFD5010AABE0030AE0
:1035E00001E1B8D60B0ACDE0020A01E100D7CBD544
:1035F0000101010E6625E96E000E6721EA6EEECF2D
:1036000000F0EDCF01F000C06AF101C06BF137ECC2
:103610002BF0B1D001016951250AD8A408D0040EBD
:10362000E124E96E000EE220EA6E050E12D00101DF
:10363000686B682B93D001016951250AD8A40BD07F
:10364000686B682B040EE124E96E000EE220EA6E3E
:10365000030EEF6E83D0080EE124E96E000EE22027
:10366000EA6E69C100F0D00E00260038F00BEF6E54
:10367000040EE124E96E000EE220EA6E060EE9D7A0
:1036800069C100F0D00E0026080EE124E96E000E9C
:10369000E220EA6E0050EF12040EE124E96E000E03
:1036A000E220EA6E080EEF6E050EE124E96E000ED0
:1036B000E220EA6EEE6AED6A51D00101050E662540
:1036C000E96E000E6721EA6EEECF00F0EDCF01F05B
:1036D00000C06AF101C06BF10101690E6C6F010E4F
:1036E0006D6F0101080E6625E96E000E6721EA6E16
:1036F000EF50E6EC14F00101050E6625E96E000EB0
:103700006721EA6E00C0EEFF01C0EDFF686B682B19
:1037100066C1E1FF67C1E2FF050EE124E96E000E1C
:10372000E220EA6EEE52ED50FF0AFF0ED8B4EF1819
:10373000D8A414D087D7FFD7040EE124E96E000E79
:10374000E220EA6EEF50030A01E164D7060A01E1C4
:1037500072D7030A95E00E0AB0E0EDD70101685177
:10376000D8B409D069C16AF166C1E9FF67C1EAFF4F
:10377000EF50CBEC08F066C1E9FF67C1EAFFEF50FC
:10378000B1EC08F00009D8B439D00101686B040E1F
:103790006625E96E000E6721EA6EEF50080AD8B47C
:1037A00016D04DEC2BF00101696F00014551FF0A65
:1037B000FF0ED8B44419D8A40AD077EC2BF066C118
:1037C000E9FF67C1EAFFEF50B3EC07F0010C66C1F7
:1037D000E1FF67C1E2FF070EE124E96E000EE2207F
:1037E000EA6EEF50D8A4A8D769C16AF166C1E9FFB3
:1037F00067C1EAFFEF50CBEC08F0BDD777EC2BF0B8
:103800000101010E6625E96E000E6721EA6E00C017
:10381000EEFF01C0EDFF000C660101016F6B746BE0
:10382000756B706B66C176F167C177F10101CD0EE2
:10383000786F060E796F0101030E7A6F7B6B5AEC7D
:1038400032F001500010D8A40BD066C1E1FF67C16F
:10385000E2FF040EE126000EE22201016E6B21D090
:1038600066C176F167C177F10101D10E786F060E5E
:10387000796F0101040E7A6F7B6B5AEC32F00150C4
:103880000010D8A4020C66C1E1FF67C1E2FF050E7B
:10389000E126000EE22201016E6B6E2B02D0E14A9E
:1038A000E22AE750200AD8B4FAD7A0D06AC1E9FFCB
:1038B0006BC1EAFFEF500101705DD8B0A7D088D08E
:1038C00001017051006E016AD8900034026E01341B
:1038D000036ED9500224E96EDA500320EA6EE1CF7C
:1038E000EEFFE2CFEDFFE7CFF3FFF3502F0AD8B49E
:1038F00029D0F3505C0AD8A477D024D001017051AC
:10390000006E016AD8900034026E0134036ED95003
:103910000224E96EDA500320EA6EE1CFEEFFE2CF37
:10392000EDFF702B020E6F6F5FD0E7CFF3FFF35008
:103930003F0AD8B404D0F350260AD8A406D0000E0B
:10394000E76A01016F6B6F2B4FD0F3502B0AD8A49D
:1039500003D0200EE76E48D0F3502E0AD8A410D022
:1039600001017005D8A40CD0E10EE96E0F0EEA6ECD
:10397000EE2A000EED22EECF74F1EDCF75F134D0CA
:10398000F3503D0AD8B4DBD7F3502F0AD8B404D093
:10399000F3505C0AD8A428D001017051006E016A6E
:1039A000D8900034026E0134036ED9500224006EA8
:1039B000DA500320016EFE0E0024E96EFF0E012096
:1039C000EA6E010EE124EE6E000EE220ED6E0CD0E8
:1039D00068C1D9FF69C1DAFF01016F5101E170D7F8
:1039E000010A8CE0030AA1E0E14AE22AE7CFD9FF0D
:1039F000D950200AD8B40AD0D950D8B407D00D0A6B
:103A0000D8B404D0D9500A0AD8A450D7000EE76A17
:103A10006CC1E9FF6DC1EAFF070EEF6E0101755140
:103A20007411D8B433D074C17AF175C17BF1DDEC77
:103A30002CF000C074F101C075F10101000E726F2D
:103A4000060E736F716B74C176F175C177F172C137
:103A500078F173C179F10101030E7A6F7B6B5AEC37
:103A600032F001500010D8A407D06CC1E9FF6DC13D
:103A7000EAFF71C1EFFF0AD0040E01017227000EA8
:103A80007323712B070E715DD8A0DDD70101705132
:103A9000D8A42ED068C1E9FF69C1EAFFEECF00F0DB
:103AA000EDCF01F000C076F101C077F10101D60E33
:103AB000786F060E796F090EE8CF7AF10EEC2DF0D3
:103AC00068C1E9FF69C1EAFFEECF00F0EDCF01F078
:103AD000090E0024E96E000E0120EA6E000EEF6A66
:103AE0006CC1E9FF6DC1EAFF010EEF6E0101702BA1
:103AF0006AC1E9FF6BC1EAFF70C1EFFF01016E51BE
:103B0000120013D00101150E016F026BE5EC05F0F8
:103B1000E8CFB2F50501B56B0501B36B0501B06BDC
:103B20000001140E676F686B1200ECD75DD1B2C54F
:103B3000E8FF23EC07F00009D8A401D001D00DD094
:103B40000501B36B070EE8CFAEF50501B56B0501B6
:103B5000B06B0501B66B010E46D1B2C5E8FF13ECA0
:103B60000AF00009D8B401D001D053D085EC33F06D
:103B700000C06BF001C06CF018D0C10E006E050ED5
:103B8000016EB3C5E8FF0024E96E000E0120EA6E65
:103B900000C1EFFF0501B32BB3C5E8FF1F0AD8A48E
:103BA00001D001D002D00501B36B0101000E666F98
:103BB000010E676FB2C5E8FFB9EC09F0006E016A4B
:103BC00001500010D8A401D001D0D7D7B2C5E8FF6A
:103BD0004CEC09F0010100510A0AD8A401D001D02F
:103BE00017D0C10E006E050E016EB3C5E8FF0024AC
:103BF000E96E000E0120EA6E000EEF6E0501B36B58
:103C0000BADA6DC005F16EC006F175DAE8CFAEF52F
:103C10004ED0B5C5E8FF0009D8B401D001D047D0D7
:103C200085EC33F000C001F101C002F16BC000F07F
:103C30006CC001F001010150025D02E10050015D24
:103C4000D8A01DD000D06BC0E8FF015D006E6CC035
:103C5000E8FF0259016E14D0FF0E006EFF0E016ED8
:103C60006BC0E8FF005C026E6CC0E8FF0158036E99
:103C700001510224006E02510320016E01D0ECD7E5
:103C800000C001F101C002F1070E025D080ED8B4B8
:103C9000015DD8A001D001D00AD001C16BF002C1F2
:103CA0006CF0020EE8CFAEF5010EE8CFB5F58ED080
:103CB0000501B16B85EC33F000C06BF001C06CF016
:103CC00000D0B2C5E8FFB1EC08F00009D8B401D0CB
:103CD00001D0F7D7B2C5E8FFB1EC08F00009D8B4BD
:103CE00001D001D03DD0B1C500F0016AD8900034B8
:103CF000026E0134036EEA0E0224E96E000E032008
:103D0000EA6EEECF03F1EDCF04F106D000C16AF107
:103D1000B2C5E8FFCBEC08F0010103C1F6FF04C116
:103D2000F7FF010E0327000E0423050EF76403D0EE
:103D30000800F55005D0F6CFE9FFF7CFEAFFEF50C6
:103D4000006F0009D8A401D001D0E0D7B2C5E8FFC8
:103D5000B3EC07F00B0EE8CFB1F5010EE8CFB5F5E7
:103D6000AEC5E8FF070AD8B401D001D02DD0AEC54A
:103D7000E8FF3BD80009D8B401D001D01AD0B1C5B2
:103D8000E8FF0B0AD8B401D001D004D0040EE8CF6C
:103D9000B5F509D0AEC5E8FF020AD8A401D001D01C
:103DA00002D00501B56B070EE8CFAEF50501B66B85
:103DB0000BD0B1C5E8FF0B0AD8B401D001D004D0B4
:103DC000040EE8CFB5F57CD70CD00BD0B5C5E8FF15
:103DD000000A01E16DD7010AC3E0050A01E170D7CD
:103DE00000D0010E00D01200A2D690D00101056FC4
:103DF0007BD0B00EE96E050EEA6EEF50FE0B0109A6
:103E0000EF6EB00EE96E050EEA6EEF50FD0BEF6E31
:103E1000010EE8CFB1F50101B70E066F050E076F71
:103E20006FC008F170C009F101010A0E0A6F0B6B37
:103E3000ADEC32F068D0B0C500F000B001D001D0D8
:103E400004D0060EE8CFB1F522D00101B70E066FFF
:103E5000050E076F6FC008F170C009F161EC15F035
:103E6000006E016A01500010D8B401D001D00CD00E
:103E7000B00EE96E050EEA6EEF50FD0B0209EF6E13
:103E8000020EE8CFB1F503D0060EE8CFB1F53BD076
:103E90003ED83BD077C024F178C025F151EC31F009
:103EA00000C068F079C024F17AC025F151EC31F0FE
:103EB00000C067F00A0EE8CFB1F525D07BD825D039
:103EC0000A0EE8CFB1F5AFC5E8FFFE0AD8B401D0BD
:103ED00001D004D0AFC5E8FF31EC07F014D0050ED7
:103EE000E8CFB1F510D00FD001010551000A81E0F3
:103EF000010AA1E0030ACCE0010AE0E0070ACAE0F7
:103F0000010ADEE0ECD7010E00D012006FD751D0CD
:103F100044D0B6C5E8FF020AD8A401D001D002D02F
:103F200021EC2BF0AFC5E8FFFE0AD8B401D001D0D8
:103F30000AD021EC2BF0AFC5E8FF31EC07F0010E01
:103F4000E8CFB6F501D00AD031D0AFC5E8FF23ECF9
:103F500007F00009D8A401D001D006D0030EE8CFA5
:103F6000B1F5030EE8CFB6F521D0B2C5E8FFB1EC4C
:103F700008F00009D8B401D001D00DD0B2C5E8FFD7
:103F800023EC07F00009D8B401D001D004D0B2C5A9
:103F9000E8FF31EC07F00AD009D0B6C5E8FF000A07
:103FA000B8E0010AD2E0020AE0E000D0000E00D042
:103FB0001200AED79ED090D0B0C500F000B201D0B4
:103FC00001D006D0060EE8CFB1F5010E91D019D080
:103FD000070EE8CFB1F5B2C5E8FF220D110EF324AC
:103FE000E8CF07F1020EF420E8CF08F167C009F12D
:103FF00068C00AF13EEC06F0E8CFAFF5010EE8CF5D
:10400000B6F574D0AFC5E8FF23EC07F00009D8B4CB
:1040100001D001D010D07AC5E8FF0009D8A401D0A2
:1040200001D009D081EC2BF000C069F001C06AF02A
:10403000020EE8CFB6F55AD0AFC5E8FF13EC0AF090
:104040000009D8B401D001D02DD085EC33F000C0E8
:104050006BF001C06CF069C02AF16AC02BF191ECE1
:104060002BF004D001010651ACEC2BF00101060E3F
:10407000666F010E676FAFC5E8FFB9EC09F0006E1F
:10408000016A01500010D8A401D001D0EBD7D3ECC5
:104090002BF000C069F001C06AF0AFC5E8FF4CEC3E
:1040A00009F019D0AFC5E8FF23EC07F00009D8A448
:1040B00001D001D010D0D3EC2BF021EC2BF0AFC508
:1040C000E8FF31EC07F0FE0EE8CFAFF5090EE8CFC0
:1040D000B1F5010E0DD00AD0B6C5E8FF000A01E126
:1040E0006BD7010A8FE0030AA7E000D0000E00D0D2
:1040F000120061D705013ED00101076B060E075D76
:10410000D8A001D001D001D032D005C176F106C1CE
:1041100077F101010751006E016AD8900034026EF8
:104120000134036EDE0E0224E96E000E0320EA6EF7
:10413000EECF00F0EDCF01F000C078F101C079F1D1
:104140000101040E7A6F7B6B5AEC32F001500010C3
:10415000D8A401D001D003D0010107510AD0010138
:10416000072B060E075DD8A001D001D0CED7060ED2
:1041700000D01200C1D77FD00101086BC10E056FBE
:10418000050E066F03D00101054B062B05C1E9FFA3
:1041900006C1EAFFEF50200AD8B401D001D0F3D70E
:1041A00005C16DF006C16EF0010EE8CFB4F556D032
:1041B0004BD001010751200AD8A401D005D00751E6
:1041C0002C0AD8A402D000D002D000D009D005C15A
:1041D000E9FF06C1EAFF000EEF6E086B082B14D052
:1041E000010107510D0AD8A401D005D007510A0AD0
:1041F000D8A402D000D002D000D006D005C1E9FF7B
:1042000006C1EAFF000EEF6E26D001010751200A19
:10421000D8B401D001D016D0B4C500F0016AD8904E
:104220000034026E0134036E6D0E0224E96E000E3E
:104230000320EA6E05C1EEFF06C1EDFF0501B42BB8
:104240000101086B08D007D001010851000AB1E054
:10425000010ADBE000D00101054B062B05C1E9FF97
:1042600006C1EAFFEF500101076F0009D8A401D091
:1042700001D09ED71200BCEF20F02A010101386B5B
:10428000396B2AC136F12BC137F101012EC1F6FF7E
:104290002FC1F7FF010E2E27000E2F23050EF76406
:1042A00003D00800F55005D0F6CFE9FFF7CFEAFFBD
:1042B000EF50336F00090101D8B4D1D2250AD8B428
:1042C0000AD0384B392B2D512C11D8A484D133511D
:1042D00003EC00F0DAD701013169326B306B6CD23C
:1042E00001012D512C11D8B406D02CC1E9FF2DC1EC
:1042F000EAFF000EEF6A38C100F039C101F0120088
:1043000001013751016E3651006E020E3627D8B0CA
:10431000372B00C0E9FF01C0EAFFEFCF32F14CD2EA
:104320000101308D49D20101302B06D0080E010168
:104330003127FE0E0101312701013751016E36513F
:10434000006E020E3627D8B0372B00C0E9FF01C03F
:10435000EAFFEECF34F1EDCF35F130A10ED035AF1D
:1043600007D0341F351F342BD8B4352B320707D074
:104370000101309130AD03D0F9D7010130910B0E1E
:10438000010131273151026E036A34C100F035C199
:1043900001F0CBEC02F00050336F3151026E036A32
:1043A00034C100F035C101F0CBEC02F004C034F1AF
:1043B00005C035F1010E3A6F3B6B01013B51355D94
:1043C00002E13A51345DD8A010D001013151026EA2
:1043D000036A3AC100F03BC101F0A5EC33F004C020
:1043E0003AF105C03BF13207E8D730A914D01AD012
:1043F0000101384B392B2D512C11D8B409D02CC1C7
:10440000E9FF2DC1EAFF200EEF6E2C4B2D2B03D0C0
:10441000200E03EC00F0010132073251800A7F0FB9
:10442000D8B0E6D730A114D00101384B392B2D512B
:104430002C11D8B409D02CC1E9FF2DC1EAFF2D0EF3
:10444000EF6E2C4B2D2B16D02D0E03EC00F012D05E
:1044500030AD10D00101384B392B2D512C11D8B46F
:1044600006D02CC1E9FF2DC1EAFF2B0EE9D72B0E98
:1044700003EC00F030B914D04DD00101384B392B8A
:104480002D512C11D8B409D02CC1E9FF2DC1EAFF60
:10449000300EEF6E2C4B2D2B03D0300E03EC00F0C2
:1044A000010132073251800A7F0FD8A033D0E5D7FF
:1044B0003AC102F03BC103F034C100F035C101F054
:1044C000CBEC02F004C000F005C001F00101315155
:1044D000026E036ACBEC02F00050326F800A760F56
:1044E000D8A002D0070E32270101384B392B2D51AD
:1044F0002C11D8B40AD03251300F2CC1E9FF2DC194
:10450000EAFFEF6E2C4B2D2B05D001013251300FFD
:1045100003EC00F001013151026E036A3A0EE96EBC
:10452000010EEA6EEE50006EEF50016ECBEC02F021
:104530000550ED6E0450EF6EEE50ED10D8A4B8D7D4
:104540000A0E0101335DD8A002D0070E3327010106
:10455000384B392B2D512C11D8B408D03351300F92
:104560002CC1E9FF2DC1EAFFEF6E3BD001013351B1
:10457000300F03EC00F089D601013251800A7E0F22
:10458000D8A015D0384B392B2D512C11D8B409D0C7
:104590002CC1E9FF2DC1EAFF200EEF6E2C4B2D2B15
:1045A00003D0200E03EC00F001013207E5D73751AC
:1045B000016E3651006E020E3627D8B0372B00C080
:1045C000E9FF01C0EAFFEFCF33F1384B392B2D5112
:1045D0002C11D8B409D02CC1E9FF2DC1EAFF33C199
:1045E000EFFF2C4B2D2B51D60101335103EC00F082
:1045F0004CD601013751016E3651006E020E36273E
:10460000D8B0372B00C0E9FF01C0EAFFEECF00F0C1
:10461000EDCF01F000C046F001C047F0D96AD95093
:10462000006E016A46C0E8FF0024026E47C0E8FF42
:104630000120036E02C0F6FF03C0F7FF050EF7640A
:1046400003D00800F55005D0F6CFE9FFF7CFEAFF19
:10465000EF500009D8B402D0D92AE1D70101315175
:10466000D95CD8B002D0D950316F0101315132BF7D
:1046700042D0FF0A3225D8A03FD0384B392B2D51DC
:104680002C11D8B409D02CC1E9FF2DC1EAFF200EAE
:10469000EF6E2C4B2D2B03D0200E03EC00F001010C
:1046A0003207E3D746C0F6FF47C0F7FF050EF764B1
:1046B00003D00800F55005D0F6CFE9FFF7CFEAFFA9
:1046C000EF500101336F0001462B000E472301011B
:1046D000384B392B2D512C11D8B409D02CC1E9FFFE
:1046E0002DC1EAFF33C1EFFF2C4B2D2B04D001016C
:1046F000335103EC00F0010131073129D8B4C5D59D
:10470000D1D72EC1F6FF2FC1F7FF050EF76403D0F6
:104710000800F55005D0F6CFE9FFF7CFEAFFEF50DC
:104720002A0AD8A412D001013751016E3651006E09
:10473000020E3627D8B0372B00C0E9FF01C0EAFFD0
:10474000EFCF31F12E4B2F2B37D02EC1F6FF2FC1DB
:10475000F7FF050EF76403D00800F55005D0F6CF3B
:10476000E9FFF7CFEAFFEF50D00F0101316F2E4B79
:104770002F2B2EC1F6FF2FC1F7FF050EF76403D0D4
:104780000800F55005D0F6CFE9FFF7CFEAFFEF506C
:10479000D96E300ED95CD8A00FD03A0ED95CD8B003
:1047A0000BD031510A0DD950F324D00F316FCAD735
:1047B00030B539D00101308901012EC1F6FF2FC17A
:1047C000F7FF010E2E27000E2F23050EF76403D0EE
:1047D0000800F55005D0F6CFE9FFF7CFEAFFEF501C
:1047E000336F000A01E17CD52A0A01E189D5010A6B
:1047F00001E196D5050A85E01E0ADAE0680A01E1C2
:1048000095D53B0A01E1B8D6070A01E18CD50B0A20
:1048100001E18FD51C0A01E1ECD6060A01E18CD535
:104820000D0A01E183D5300E0101335DD8A00CD013
:104830003A0E335DD8B008D0308532510A0D33516D
:10484000F324D00F326FB8D70101384B392B2D51DB
:104850002C11D8A4C0D6335103EC00F016D52D513D
:104860002C11D8B406D02CC1E9FF2DC1EAFF000EEF
:10487000EF6A38C100F039C101F012009EBA9DAA5A
:1048800009D1AB50060BD8B405D0AB98AB88050E58
:10489000E8CF4AF0AECF48F04C0EE96E000EEA6E5B
:1048A000EF50FE0BEF6E4A0EE96E000EEA6EEF500F
:1048B000010A23E0030A2FE0010A3EE0070A70E044
:1048C000010A01E190D002C349F000014B6B48C0DE
:1048D000E8FFC00AD8A402D0030E43D048C0E8FFC6
:1048E000410AD8A484D04C0EE96E000EEA6EEF5057
:1048F000FE0B0109EF6E020E34D04C0EE96E000E75
:10490000EA6EEF50FE0B0109EF6E48C0E8FF0D0A9A
:10491000D8A46DD035D04C0EE96E000EEA6EEF5083
:10492000FE0B0109EF6E48C0E8FF540AD8A402D07C
:10493000010E17D0050E15D04C0EE96E000EEA6E72
:10494000EF50FE0B0109EF6E48C0E8FFDB0AD8A468
:104950000BD04C0EE96E000EEA6EEF50FE0BEF6EC0
:10496000040EE8CF4AF043D048C0E8FFC00AD8A4FC
:104970003ED04B0EE96E000EEA6EEF50D8B409D06F
:104980004C0EE96E000EEA6EEF50FD0B0209EF6E61
:104990002ED04C0EE96E000EEA6EEF50FE0BF7D7EC
:1049A0004C0EE96E000EEA6EEF50FE0B0109EF6E41
:1049B000030EE8CF4AF048C0E8FFDC0AD8A402D0D2
:1049C000C00E06D048C0E8FFDD0AD8A404D0DB0E34
:1049D000E8CF48F00CD04C0EE96E000EEA6EEF50B6
:1049E000FE0BEF6E02D049C002F300014A6B4CC0CF
:1049F00000F000A030D00301022BFA0E02C300F039
:104A0000005CD8B0026B00C300F0020EE96E030E2A
:104A1000EA6EEF500018D8B413D000014B2B040EEF
:104A2000006E030E016E020EE96E030EEA6EEF5089
:104A30000024E96E000E0120EA6E48C0EFFF0BD0A3
:104A400049C002F300014A6B4C0EE96E000EEA6E9B
:104A5000EF50FD0BEF6E4CC000F000A21BD04C0ECF
:104A6000E96E000EEA6EEF50FD0BEF6E040E006E65
:104A7000030E016E490EE96E000EEA6EEF5000243F
:104A8000E96E000E0120EA6E02C3EFFF0301012B65
:104A900000014A6B9EA812009DA81200000EE96E4C
:104AA000040EEA6EEF50D8B445D0040E006E016ECD
:104AB000010EE96E040EEA6EEF500024E96E000E5E
:104AC0000120EA6EEF50E8CF48F048C0E8FFC00A86
:104AD000D8A412D0DB0EE8CF48F0040E006E016EB1
:104AE000010EE96E040EEA6EEF500024E96E000E2E
:104AF0000120EA6EDC0E16D048C0E8FFDB0AD8A41D
:104B000013D0DB0EE8CF48F0040E006E016E010EEC
:104B1000E96E040EEA6EEF500024E96E000E0120EB
:104B2000EA6EDD0EEF6E03D004010007012B48C0D2
:104B3000ADFF12009D9803C400F000A008D0030E42
:104B4000E96E040EEA6EEF50FE0BEF6E1200C00E1F
:104B5000AD6E1200000E1BD900014A6B00014C6BB8
:104B60000301006B016B036B026B05017B6B9E9A6B
:104B70009D8A9D98200EAC6E900EAB6E070EAF6EA8
:104B8000F28EF28C1200FA0E00C400F0005CD8A085
:104B90009DB8000C010C0601010EE8CF7BF5E96E13
:104BA000030EEA6EEF50D8B4000C00C303F3030108
:104BB000032BFA0E03C300F0005CD8B0036B040EA5
:104BC000006E030E016EE96EEA6EEF500024E96E8E
:104BD000000E0120EA6EEF50410AD8A41AD063D823
:104BE000030EE96E040EEA6EEF50FE0B0109EF6E44
:104BF000040EE8CF00F40401026B05017B6B4F0E3D
:104C000075D84B0E73D80D0E71D80A0E6FD8B4D864
:104C1000000C08C1E9FF09C1EAFFEF6A010C7BC57E
:104C2000E8FF0009040E006ED8B414D0030E016E24
:104C30000301032B03050024E96E000E0120EA6E38
:104C4000EFCFD9FFFA0E03C300F0005CD8A00ED05E
:104C5000036B0CD0040E016E0401022B020500242C
:104C6000E96E000E0120EA6EEFCFD9FFD950120095
:104C7000400101014351016E4251006E4207D8A02C
:104C800043070110D8B40AD0CADF40C1E9FF41C1CF
:104C9000EAFFEF6E0101404B412BEBD742C100F020
:104CA00043C101F012009D9A010EE96E030EEA6EF7
:104CB000EF50D8B411D0040E006E030E016EE96AF5
:104CC000EA6EEF500024E96E000E0120EA6EEF500C
:104CD000E8CF00F3030101079D8A1200C101C4C19E
:104CE00000F40401026B05017B6B1200D96E7BC5D9
:104CF000E8FF0009040E006ED8B414D0030E016E54
:104D00000301032B03050024E96E000E0120EA6E67
:104D1000D9CFEFFFFA0E03C300F0005CD8A0120059
:104D2000036B1200040E016E0401022B0205002425
:104D3000E96E000E0120EA6ED9CFEFFF1200C1012B
:104D4000C1C1E1FFC2C1E2FF0101C451016EC35103
:104D5000006EC307D8A0C4070110D8B41200E250F7
:104D6000016EE150006EE14AE22A00C0E9FF01C095
:104D7000EAFFEF50BBDFE8D70401026B016B03C40D
:104D800000F000B002D0C00EAD6E9D8812009DB83C
:104D900012000401006B026B016B036B12006A01CD
:104DA000E96A030EEA6EEF5001016A27000E6B23D9
:104DB0006A4B6B2B6B5DF90ED8B46A5DD8A005D039
:104DC0006A51060FE8CF03F302D06AC103F3010E64
:104DD000E8CF7BF51200A801A8C102F405017B6BA6
:104DE000120012009D9A020EE96E030EEA6EEFCFDA
:104DF000D9FF9D8A010EE96E030EEA6EEF50D8B41A
:104E00001DD0D95000C300F0005CD8B00FD0FA0E0E
:104E1000006E016AD950005E000E015AE96A030E65
:104E2000EA6EEF500026000E01221200D95000C396
:104E300000F0016A005E000E015A1200F80E006ECA
:104E4000016A1200110196D00101150E406F010E8A
:104E5000416F01011C0E426F436B39EC26F053EC9D
:104E600026F00101150E316F010E326F62D901017A
:104E70001551010A1611D8B401D006D019C1E8FFA6
:104E8000060AD8B402D000D007D000D01AC1E8FF7B
:104E9000040AD8B402D000D002D000D002D0000E54
:104EA00068D013C1E1FF14C1E2FF11C1D9FF12C1E3
:104EB000DAFF01011B51020A1C11D8A401D001D054
:104EC00003D0000EE76E0FD001011B51010A1C1127
:104ED000D8A401D001D003D0010EE76E04D0020E99
:104EE000E76E000E46D07BC0E8FF01012D630AD0BB
:104EF00000D07C0EE96E000EEA6EEF502E6302D0F9
:104F000000D001D009D07D0EE96E000EEA6EEF50A0
:104F10002F6302D000D001D009D07E0EE96E000EC2
:104F2000EA6EEF50306302D000D002D000D01FD024
:104F30001D0E006E010E016E00C0E9FF01C0EAFF08
:104F4000D9CFE1FFDACFE2FF060ED2EC33F0060E46
:104F5000D924E96E000EDA20EA6E23C1EEFF24C1E7
:104F6000EEFF25C1EEFF26C1EEFF010E02D0000EBE
:104F700000D0120069D71101DAD011C1D9FF12C1D6
:104F8000DAFF0101010E146F156B0101000E166F9F
:104F9000080E176F060EE8CF18F1040EE8CF19F1CE
:104FA00001011305D8A401D001D017D00101010ED1
:104FB0001A6F1B6BFF0EE8CF26F1FF0EE8CF27F12B
:104FC000FF0EE8CF28F1FF0EE8CF29F1FF0EE8CF62
:104FD0002AF1FF0EE8CF2BF113D00101020E1A6F58
:104FE0001B6BD9CF00F0DACF01F000C0E9FF01C0A0
:104FF000EAFF260EE16E010EE26E060ED2EC33F0F1
:105000007FC01CF180C01DF181C01EF182C01FF164
:1050100083C020F184C021F17BC022F17CC023F148
:105020007DC024F17EC025F185C000F0060ED92494
:10503000E96E000EDA20EA6EEF50016E01010150B8
:1050400022190014D8B401D010D086C000F0070E89
:10505000D924E96E000EDA20EA6EEF50016E01509D
:1050600023190014D8B402D000D011D000D087C0CA
:1050700000F0080ED924E96E000EDA20EA6EEF5037
:10508000016E015024190014D8B402D000D011D000
:1050900000D088C000F0090ED924E96E000EDA2095
:1050A000EA6EEF50016E015025190014D8B402D0F9
:1050B00000D002D000D009D089C02CF18AC02DF1D7
:1050C0008BC02EF18CC02FF110D0060ED924E96EC2
:1050D000000EDA20EA6EEECF2CF1EECF2DF1EECFFE
:1050E0002EF1EDCF2FF1ED52ED520101140E316F83
:1050F000010E326F1ED80101260EC16F010EC26F64
:10510000060EE8CFC3F101011C0EC46FC56B6FEC36
:1051100026F00101140EC16F010EC26F01011C0EB9
:10512000C36FC46BA0EC26F0BCEC26F0120025D7B0
:1051300031014ED031C1E9FF32C1EAFFEECF00F0BC
:10514000EDCF01F000C0C3F101C0C4F1E9EC2BF0D8
:1051500031C1E9FF32C1EAFF00C0EEFF01C0EDFF3F
:105160000101020E3125E96E000E3221EA6EEECF0A
:1051700000F0EDCF01F000C0C3F101C0C4F1E9ECD3
:105180002BF00101020E3125E96E000E3221EA6E8C
:1051900000C0EEFF01C0EDFF060E3125E96E000EE6
:1051A0003221EA6EEECF00F0EDCF01F000C0C3F186
:1051B00001C0C4F1E9EC2BF00101060E3125E96EC6
:1051C000000E3221EA6E00C0EEFF01C0EDFF1200BA
:1051D000B1D7060101012B0E406F010E416F010195
:1051E000140E426F436B39EC26F0F00E006E010195
:1051F0002B15400AD8A4B5D02BC100F00F0E001615
:10520000D8900036D8900034EC0F0E6F150E0E5D5E
:10521000D8B0A7D00E51D8B40CD00101170E406FF2
:10522000010E416F01010E510101426F436B39ECD8
:1052300026F0350EE96E010EEA6EEECF11F1EDCFDC
:1052400012F10101356B366B01012B0EC16F010E9E
:10525000C26F0101140EC36FC46B52EC2CF0001C22
:10526000026E011C036E02C013F103C014F10101B0
:105270000E51D8B415D00101170EC16F010EC26FC7
:1052800001010E510101C36FC46B52EC2CF0001CE4
:10529000026E011C036E02C015F103C016F103D0AB
:1052A0000101156B166B0101130EC16F010EC26F68
:1052B0000101040EC36FC46B52EC2CF000C00FF15F
:1052C00001C010F101012B0EC16F010EC26FB9D8E0
:1052D00001011051121902E10F511119D8A441D046
:1052E000F00E006E2B15400AD8A43BD006C1E1FF9A
:1052F00007C1E2FFE250E110D8B40CD0E1CFE9FFE2
:10530000E2CFEAFF3BC1EEFF3CC1EEFF3DC1EEFF45
:105310003EC1EEFF0101060E0825E96E000E0921CF
:10532000EA6E37C1EEFF38C1EEFF39C1EEFF3AC178
:10533000EEFF0AC1E9FF0BC1EAFF34C1EFFF0E51D6
:105340002D5D006E2E51D8A02E05016EEC0E0024AE
:105350000CC1E9FF0DC1EAFFEE6EFF0E0120ED6EFC
:10536000010C53EC26F0000CA801450EE8CFADF17E
:105370000101AE6B140EAB25E8CFAFF1000EAC21EE
:10538000E8CFB0F10001402B000E412340C0B1F145
:1053900041C0B2F10101B36BB46B640EE8CFB5F15B
:1053A000AAC1B6F1B76BB86B7BC0B9F17CC0BAF1DA
:1053B0007DC0BBF17EC0BCF1060EA825E96E000ED3
:1053C000A921EA6EEECFBDF1EECFBEF1EECFBFF177
:1053D000EDCFC0F1ED52ED520101AD0EC16F010EE6
:1053E000C26F2FD80101AD0EC16F010EC26F010156
:1053F000140EC36FC46B52EC2CF000C0B7F101C0A7
:10540000B8F1A8C1C1F1A9C1C2F10101C36B010189
:10541000140EAB25E8CFC4F1000EAC21E8CFC5F1E6
:105420006FEC26F00101AD0EC16F010EC26F0101DC
:10543000140EC36FC46BA0EC26F0006A016A120060
:10544000C1010101020EC125E96E000EC221EA6E02
:10545000EECF00F0EDCF01F000C0C3F101C0C4F108
:10546000E9EC2BF00101020EC125E96E000EC2210C
:10547000EA6E00C0EEFF01C0EDFF040EC125E96E2B
:10548000000EC221EA6EEECF00F0EDCF01F000C0B9
:10549000C3F101C0C4F1E9EC2BF00101040EC125F8
:1054A000E96E000EC221EA6E00C0EEFF01C0EDFF02
:1054B0000A0EC125E96E000EC221EA6EEECF00F0A1
:1054C000EDCF01F000C0C3F101C0C4F1E9EC2BF055
:1054D00001010A0EC125E96E000EC221EA6E00C06C
:1054E000EEFF01C0EDFF12000AD005017A6B050145
:1054F000796B0B0E5FEC00F0010E00D01200F5D7B7
:1055000066019ED079C500F000A001D001D003D083
:10551000006A016A94D0200E0101776F786B66C132
:10552000E9FF67C1EAFFEF50D8A401D001D005D050
:10553000FF0E006EFF0E016E82D066C17AF167C168
:105540007BF1DDEC2CF000C066F101C067F171D099
:1055500077C17AF178C17BF10101680E7C6F010E91
:105560007D6F0F0EE8CF7EF1A00EF9EC01F0680E12
:10557000E96E010EEA6EEF50D8A401D001D038D008
:1055800066C17AF167C17BF12FEC33F00050010165
:10559000796F0D0E795DD8A001D001D002D00C0E2C
:1055A000796F66C17AF167C17BF101016B0E7C6F87
:1055B000010E7D6F0101795101017E6F7F6BEDEC72
:1055C00031F001500010D8A401D001D00BD005015A
:1055D0007A2B690EE96E010EEA6EEECF00F0EDCF88
:1055E00001F02DD00F0E01017727000E782321D076
:1055F00068C1E8FF040AD8A401D001D015D0010188
:105600006A51FF0AFF0ED8B46919D8B401D001D08D
:1056100009D0690EE96E010EEA6EEECF77F1EDCF9B
:1056200078F101D007D005D0FF0E006EFF0E016E9D
:1056300006D08ED7FF0E006EFF0E016E00D0120056
:1056400061D713D00501786B790EE96E050EEA6E0D
:10565000EF50FE0BEF6E7AC5E8FF0009D8B401D019
:1056600001D002D005017A071200ECD76A0114D0EC
:105670006AC144F06BC145F06AC181F16BC182F12E
:10568000A00E0AEC01F0006E016A01500010000E3D
:10569000D8B4010E00D01200EBD728D0CEEC01F028
:1056A00001016A6F0001442B000E452301016A517C
:1056B000030AD8A401D001D009D0CEEC01F0010139
:1056C0006A6F0001442B000E45230CD001016A5182
:1056D000040AD8A401D001D005D0FF0EE8CF44F0D1
:1056E000E8CF45F001016A5100D01200D7D708D0A9
:1056F000E0EC01F044C000F045C001F000D0120021
:10570000F7D70DD0790EE96E050EEA6EEF50FE0B5D
:105710000109EF6E200E006E016A00D01200F2D770
:105720002A0119D02AC144F02BC145F02AC178F5CD
:1057300005013F0E78172AC185F12BC186F1A00E15
:1057400070EC00F0006E016A01500010000ED8B439
:10575000010E00D01200E6D725D001012A6F2A5190
:1057600070EC01F00009D8B401D001D002D0000ED5
:1057700018D00501782B0001442B000E4523400E64
:1057800078C500F0005CD8A001D001D008D00BD8BB
:1057900044C085F145C086F1A00E70EC00F0010E0A
:1057A00000D01200DAD713D00501786BAFEC01F00E
:1057B00000D0A00E49EC02F00009D8A401D001D01D
:1057C000F8D744C000F045C001F000D01200ECD77B
:1057D000C30114D0C3C1C5F1C4C1C6F1C60EE96E80
:1057E000010EEA6EEFCFC7F1C5C1C6F1C7C1C5F161
:1057F000C5C100F0C6C101F000D01200EBD7AA016C
:105800004FD0AAC1AFF1ABC1B0F1ACC1B1F1ADC1E4
:10581000B2F10101AF0EB36F010EB46F030EB325E9
:10582000E96E000EB421EA6EEFCFAEF1B3C1E9FF2D
:10583000B4C1EAFF030EB325E16E000EB421E26E9F
:10584000EFCFE7FFB3C1E9FFB4C1EAFFAEC1EFFF9D
:10585000020EB325E96E000EB421EA6EEFCFAEF171
:10586000010EB325E16E000EB421E26E020EB325E7
:10587000E96E000EB421EA6EE7CFEFFF010EB3250B
:10588000E96E000EB421EA6EAEC1EFFFAFC100F0C9
:10589000B0C101F0B1C102F0B2C103F000D01200FA
:1058A000B0D7C10188D00101C56BC66BC76BC86B8F
:1058B000D890C431CA6FC331C96FC1C1CBF1C2C165
:1058C000CCF11BD00101CC51016ECB51006E020E08
:1058D000CB27D8B0CC2B00C0E9FF01C0EAFFEECF48
:1058E00000F0EDCF01F0026A036A0050C5270150B5
:1058F000C6230250C7230350C8230101CA51016EB9
:10590000C951006EC907D8A0CA0701500010D8A419
:1059100001D001D0D7D7C3A101D001D00ED0CBC1C7
:10592000E9FFCCC1EAFFEF500101C527010ED8B055
:10593000C627D8B0C727D8B0C8272BD00101CD5172
:10594000046ECE51056E066A076AFF0EC515006E1D
:10595000FF0EC615016E000EC715026E000EC815AB
:10596000036E04C0E8FF0024086E05C0E8FF0120B4
:10597000096E06C0E8FF02200A6E07C0E8FF032098
:105980000B6E08C0C5F109C0C6F10AC0C7F10BC053
:10599000C8F1C7C1CDF1C8C1CEF10101CE51CD11C1
:1059A000D8A401D001D0CAD70101C51D006EC61D03
:1059B000016E00D0120077D77A012ED07AC17DF126
:1059C0007BC17EF117D0610E01017C5DD8A007D0AC
:1059D00000D07B0E7C5DD8B002D000D002D000D0C9
:1059E00006D07DC1E9FF7EC1EAFFE00EEF2601018E
:1059F0007D4B7E2B7DC1E9FF7EC1EAFFEF500101A7
:105A00007C6F0009D8A401D001D0DDD77AC100F0A5
:105A10007BC101F000D01200D1D776012FD078C120
:105A20007DF179C17EF176C17BF177C17CF119D02E
:105A30007DC1F6FF7EC1F7FF7BC1E9FF7CC1EAFFB4
:105A4000050EF76403D00800F55005D0F6CFE1FF4E
:105A5000F7CFE2FFE750EF6E01017B4B7C2B7D4BD4
:105A60007E2B01017A077A29D8A401D001D0E0D792
:105A700076C100F077C101F000D01200D0D7060146
:105A80000101180E406F010E416F0101080E426FB7
:105A9000436B39EC26F01A0EE96E010EEA6EEECF7A
:105AA00012F1EDCF13F101011A6B1B6B0101180EFE
:105AB000C16F010EC26F0101080EC36FC46B52ECBF
:105AC0002CF0001C026E011C036E02C014F103C016
:105AD00015F10AC1E1FF0BC1E2FFF80EE72608C18C
:105AE00040F109C141F1E7500101426F436B39ECCC
:105AF00026F008C1C1F109C1C2F10AC1E9FF0BC119
:105B0000EAFFEF500101C36FC46B52EC2CF0001C94
:105B1000026E011C036E02C016F103C017F10101F1
:105B2000140EC16F010EC26F0101040EC36FC46B6E
:105B300052EC2CF000C010F101C011F10101180E5F
:105B4000406F010E416F86D806C1E9FF07C1EAFF29
:105B500018C1EFFF0CC1E9FF0DC1EAFF1CC1EEFF48
:105B60001DC1EDFF0EC1E9FF0FC1EAFF1EC1EEFF2F
:105B70001FC1EDFF01011351111902E1125110195A
:105B8000000ED8B4010E120006010101116B08C10C
:105B900010F1126B136B0CC114F10DC115F10EC194
:105BA00016F10FC117F10101180E466F010E476F74
:105BB00009C148F10AC149F101010B5101014A6FC4
:105BC0004B6BF7EC32F00101100E406F010E416F8C
:105BD00041D80101100EC16F010EC26F01010B51BE
:105BE000006E016A080E0024E8CFC3F1000E012008
:105BF000E8CFC4F152EC2CF000C012F101C013F157
:105C000006C1A8F107C1A9F1010EE8CFAAF101016F
:105C10000B51006E016A080E0024E8CFABF1000EB4
:105C20000120E8CFACF1B5EC29F00101100EC16FF5
:105C3000010EC26F01010B51006E016A080E0024B3
:105C4000E8CFC3F1000E0120E8CFC4F1A0EC26F0AC
:105C5000BCEF26F00101040E4025E96E000E412143
:105C6000EA6EEECF00F0EDCF01F000C0C3F101C04D
:105C7000C4F1E9EC2BF00101040E4025E96E000EA1
:105C80004121EA6E00C0EEFF01C0EDFF060E402587
:105C9000E96E000E4121EA6EEECF00F0EDCF01F08B
:105CA00000C0C3F101C0C4F1E9EC2BF00101060E04
:105CB0004025E96E000E4121EA6E00C0EEFF01C0F2
:105CC000EDFF020E4025E96E000E4121EA6EEECF97
:105CD00000F0EDCF01F000C0C3F101C0C4F1E9EC68
:105CE0002BF00101020E4025E96E000E4121EA6E03
:105CF00000C0EEFF01C0EDFF120005017C6BAAECB5
:105D000025F071EC30F08AEF05F00101006B002BFB
:105D100001010051D8B421EF0AF0006BD2D001018B
:105D20005D0E066F000E076F0101010E086F010E78
:105D3000096FCCEC25F0006E016A015000100101E2
:105D4000D8B4E7D7006B002B0151D8A402D0020EC3
:105D50003CD001010151060AD8A402D0050E35D06D
:105D600053EC26F0D5D70101006B88EC30F0000928
:105D7000D8B4CED731D00101020E066F010E076FE5
:105D800001015D0E086F000E096F0101010E0A6F1F
:105D9000010E0B6F0101570E0C6F000E0D6FEAEC38
:105DA00028F0006E016A01500010D8B418D001012B
:105DB000006B002B0105D8A402D0030E06D0010110
:105DC0000151060AD8A404D0060EE8CF7CF5A0D76E
:105DD0000101006B53EC26F005017C6B99D753EC65
:105DE00026F0FAD701015D0E066F000E076F57C04F
:105DF00008F158C009F123EC0AF0006E016A015065
:105E00000010D8B402D005017C6B0101006B80D773
:105E100005017C6B0001000E585D2A0ED8B4575D59
:105E2000D8B02ED00101010E066F010E076F0101DF
:105E30007D0E086F050E096F0101570E0A6F000EE7
:105E40000B6F0101590E0C6F000E0D6F01015B0EFF
:105E50000E6F000E0F6F40EC2DF0006E016A0150C6
:105E60000010D8B40BD001010151080AD8A406D003
:105E7000006B002B040EE8CF7CF502D005017C6B93
:105E800053EC26F045D7C3EC25F00009D8B440D731
:105E900001015D0E066F000E076F0101086B010125
:105EA0007D0E096F050E0A6F57C00BF159C00CF13A
:105EB0005AC00DF15BC00EF15CC00FF1C5EC2DF0C6
:105EC0008BD77CC5E8FF000A01E129D7010A01E16F
:105ED00026D7030A01E14FD7010A9AE0070AD3E067
:105EE000010A01E140D7030A01E17CD788EF2EF0D7
:105EF00037D0F00E83160F0E9512959A9598929AB8
:105F0000839A8398809A7EEC18F0F00E9516F00E26
:105F100083168382808A00F000F0809A81EC18F06A
:105F2000F00E83168382808A00F000F0809A84EC61
:105F300018F0F00E83168382808A00F000F0809AB9
:105F40000F0E9512280E0DD8080E0BD80C0E09D87E
:105F5000010E07D8130E05D8800E03D800D012000A
:105F6000C8D72CD001012A6F00D029D80009D8A4A5
:105F700001D001D0FAD7959A9598F00E9516F00EAB
:105F8000831601012A390F0B8312839A839800F03C
:105F900000F0808A00F000F0809AF00E83160F0E59
:105FA000006E00502A15831200F000F0808A00F085
:105FB00000F0809A0F0E951200D01200D3D723D094
:105FC000959A9598838A839800F000F0808A00F073
:105FD00000F083A601D001D00BD0809A00F000F031
:105FE000808A00F000F0809A839A010E0BD00AD0CC
:105FF000809A00F000F0808A00F000F0809A839A86
:10600000000E00D01200DCD72A0114D006D0010106
:106010002C5132D801012A4B2B2B2AC1E9FF2BC16D
:10602000EAFFEF5001012C6F0009D8A401D001D084
:10603000EED71200EBD72A011ED006D001012C5159
:106040001BD801012A4B2B2B2AC1F6FF2BC1F7FFCE
:10605000050EF76403D00800F55005D0F6CFE9FF30
:10606000F7CFEAFFEF5001012C6F0009D8A401D04F
:1060700001D0E4D71200E1D733D001012D6F00D059
:106080009EDF0009D8A401D001D0FAD7959A95983F
:10609000F00E9516F00E83160F0E006E2DC101F056
:1060A000013A0F0E01160050011483128388839A5F
:1060B00000F000F0808A00F000F0809AF00E831665
:1060C0000F0E006E010100502D15831200F000F03C
:1060D000808A00F000F0809A0F0E951200D0120016
:1060E000CCD715D00501776BFF0EE8CF4DF0FF0E32
:1060F000E8CF4EF0FF0EE8CF4FF0FF0EE8CF50F0A4
:10610000FF0EE8CF51F0FF0EE8CF52F01200EAD7B1
:1061100053D04AD00101070E116F010E126F010119
:10612000060E136F010E146F23EC27F0006E016A48
:1061300001500010D8A401D001D001D03AD0010103
:1061400006510009D8A401D001D015D007C14DF0E7
:1061500008C14EF009C14FF00AC150F00BC151F017
:106160000CC152F00DC153F00EC154F00FC155F0E7
:1061700010C156F01ED0010EE8CF77F5C3EC25F024
:106180000009D8B401D001D00CD00101070E116F65
:10619000010E126F0101136BBCEC27F00501776B48
:1061A00002D0000E08D005D077C5E8FF000AB2E0A3
:1061B000E5D7010E00D01200ACD7000119D000C104
:1061C000E9FF01C1EAFFEECF06F1EECF07F1EECF16
:1061D00008F1EDCF09F1ED52ED520101000E116F02
:1061E000010E126F010EE8CF13F1BCEC27F0120084
:1061F000E6D7000154D000C1E9FF01C1EAFF000168
:106200005351EE1808E15451EE1805E15551EE18BE
:1062100002E15651EE18D8A401D02ED0890EE96EB5
:10622000000EEA6EEF5053C000F000620CD000D0B8
:106230008A0EE96E000EEA6EEF5054C000F0006264
:1062400002D000D001D00BD08B0EE96E000EEA6EAA
:10625000EF5055C000F0006202D000D001D00BD04A
:106260008C0EE96E000EEA6EEF5056C000F0006230
:1062700002D000D001D001D002D000D00DD04D0E00
:10628000E96E000EEA6E02C1E1FF03C1E2FF060EF5
:10629000D2EC33F0010E02D0000E00D01200ABD7CA
:1062A000240103D00101244B252B24C1F6FF25C175
:1062B000F7FF050EF76403D00800F55005D0F6CFC0
:1062C000E9FFF7CFEAFFEF50200AD8B4EBD724C19B
:1062D000F6FF25C1F7FF050EF76403D00800F5505F
:1062E00005D0F6CFE9FFF7CFEAFFEF50090A010129
:1062F000D8B4D9D7276B286B266B24C1F6FF25C1EC
:10630000F7FF050EF76403D00800F55005D0F6CF6F
:10631000E9FFF7CFEAFFEF502D0AD8A402D0262BD1
:1063200013D024C1F6FF25C1F7FF050EF76403D093
:106330000800F55005D0F6CFE9FFF7CFEAFFEF50A0
:106340002B0AD8A403D00101244B252B24C1F6FF2E
:1063500025C1F7FF050EF76403D00800F55005D0FE
:10636000F6CFE9FFF7CFEAFFEF50B3EC33F0D8A058
:1063700025D00A0E026E036A27C100F028C101F081
:10638000A5EC33F024C1F6FF25C1F7FF050EF76435
:1063900003D00800F55005D0F6CFE9FFF7CFEAFFAC
:1063A000EF500424006E000E0520016ED00E002474
:1063B0000101276FFF0E0120286FC6D7010126516A
:1063C00027C100F028C101F0D8B41200001E011E40
:1063D000002AD8B4012A12007A0101017F51016E0E
:1063E0007E51006E7E07D8A07F070110D8B45ED022
:1063F0007AC1F6FF7BC1F7FF050EF76403D00800F2
:10640000F55005D0F6CFE9FFF7CFEAFFEF500009CE
:10641000D8B422D07CC1F6FF7DC1F7FF050EF7642A
:1064200003D00800F55005D0F6CFE9FFF7CFEAFF1B
:10643000EF50006E7AC1F6FF7BC1F7FF050EF764DF
:1064400003D00800F55005D0F6CFE9FFF7CFEAFFFB
:10645000EF500018D8B424D07AC1F6FF7BC1F7FF03
:10646000050EF76403D00800F55005D0F6CFE9FF1C
:10647000F7CFEAFFEF50006E016A7CC1F6FF7DC1E5
:10648000F7FF050EF76403D00800F55005D0F6CFEE
:10649000E9FFF7CFEAFFEF50005E000E015A12004D
:1064A00001017A4B7B2B7C4B7D2B97D7006A016ACD
:1064B0001200760176C102F077C103F078C1F3FFD4
:1064C00079C1F4FF01017B51016E7A51006E7A07A8
:1064D000D8A07B070110D8B43CD0F3CFF6FFF4CF9F
:1064E000F7FF010EF326000EF422050EF76403D029
:1064F0000800F55005D0F6CFE9FFF7CFEAFFEF50DF
:10650000016E02C0F6FF03C0F7FF010E0226000E67
:106510000322050EF76403D00800F55005D0F6CF2E
:10652000E9FFF7CFEAFFEF50006E0150005C010178
:106530007C6F7D6BD8A07D0700BE7D0701BE7D2BE3
:106540007D517C11D8B4BED77CC100F07DC101F073
:106550001200006A016A1200060106C1D9FF07C1D4
:10656000DAFF01010B510A11D8B425D00A07D8A0CF
:106570000B0708C1F6FF09C1F7FF010E0827000E3F
:106580000923DA50016ED950006ED94ADA2A00C0C8
:10659000E9FF01C0EAFF050EF76403D00800F550DB
:1065A00005D0F6CFE1FFF7CFE2FFE750EF6EEF50F7
:1065B000D8A4D7D701010B51016E0A51006E0A070A
:1065C000D8A00B070110D8B40CD0DA50016ED95006
:1065D000006ED94ADA2A00C0E9FF01C0EAFFEF6A7B
:1065E000E9D706C100F007C101F01200460148C119
:1065F000F3FF49C1F4FF46C1D9FF47C1DAFF0101EA
:106600004B51016E4A51006E4A07D8A04B0701104A
:10661000D8B41FD0F3CFF6FFF4CFF7FF010EF32667
:10662000000EF422DA50016ED950006ED94ADA2AEF
:1066300000C0E9FF01C0EAFF050EF76403D00800BF
:10664000F55005D0F6CFE1FFF7CFE2FFE750EF6E50
:10665000D6D746C100F047C101F012007A017AC1D5
:10666000F3FF7BC1F4FFF3CFF6FFF4CFF7FF010E8A
:10667000F326000EF422050EF76403D00800F5504F
:1066800005D0F6CFE9FFF7CFEAFFEF500009D8A415
:10669000EAD701017A51F35C006E7B51F458016E28
:1066A000FF0E0024006EFF0E0120016E120022D0AA
:1066B0000101016F17D00101040E006F0CD0010120
:1066C000500E026F03D00101026B022B01D000D0EB
:1066D0000101022FFCD7010100070029D8A401D035
:1066E00001D0EDD7010101070129D8A401D001D0C3
:1066F000E2D71200DDD75E0ED66EF80ED76E070E0B
:10670000D56ED58EF284F28A120042C000F043C0EA
:1067100001F01200F2A41200F80ED76E5E0ED66ED3
:106720000001422B000E43238978F2941200EFCF30
:1067300000F0EE2AEFCF01F0000EEE22EFCF02F0D4
:10674000EE22EFCF03F0EE22120002500002F3CF50
:1067500004F0F4CF05F00102F350052603500002C7
:10676000F35005261200D96E3A0ED95CD8B006D087
:10677000300ED95CD8A002D0D8801200D890120078
:106780000900F5CFEEFFEA50E262FAD7E950E16284
:10679000F7D71200EE6AEA50E262FCD7E950E162F4
:0E67A000F9D71200EECFE6FFE82EFCD7000C72
:020000040030CA
:04000000FFFAFCFE09
:020000040000FA
:00000001FF
